:020000040002F8
:10600000D0510020C1630200C9630200CB630200CB
:10601000CD630200CF630200D163020000000000E4
:10602000000000000000000000000000D363020038
:10603000D563020000000000D7630200D9630200AC
:1060400041670200DB630200E16A0200DB630200D9
:10605000DB630200DB63020079650200DB630200A0
:10606000DB630200DB630200DB630200DB63020030
:10607000DB630200DB630200DB630200DB63020020
:10608000DB63020099670200DB630200DB6302004E
:10609000BD670200DB630200C1670200DB63020030
:1060A000DB630200DB630200DB630200DB630200F0
:1060B000DB630200DB630200000000000000000060
:1060C000DB630200DB630200DB630200DB630200D0
:1060D000DB630200DB630200DB6302000000000000
:1060E00000000000000000000000000000000000B0
:1060F00000000000000000000000000000000000A0
:10610000000000000000000000000000000000008F
:10611000000000000000000000000000000000007F
:10612000000000000000000000000000000000006F
:10613000000000000000000000000000000000005F
:10614000000000000000000000000000000000004F
:10615000000000000000000000000000000000003F
:10616000000000000000000000000000000000002F
:10617000000000000000000000000000000000001F
:10618000000000000000000000000000000000000F
:1061900000000000000000000000000000000000FF
:1061A00000000000000000000000000000000000EF
:1061B00000000000000000000000000000000000DF
:1061C00000000000000000000000000000000000CF
:1061D00000000000000000000000000000000000BF
:1061E00000000000000000000000000000000000AF
:1061F000000000000000000000000000000000009F
:10620000DFF80CD000F07AF900480047C5A402007E
:10621000D051002030B450E8012F93B2C4892344F8
:106220008489A34228BF1B1B0489A34202BFBFF37A
:106230002F8F002007E0C3EA020340E80134002C5E
:10624000E9D14FF001000A6030BC704750E8012FDF
:10625000C2EA024240E801210029F7D1704730B478
:1062600050E8022F1FFAA2F3C488A34202BFBFF373
:106270002F8F00200DE0C48923448489A34228BFC6
:106280001B1BC2EA034340E80234002CE8D14FF064
:1062900001000A6030BC704750E8022FC2EA224277
:1062A00040E802210029F7D17047034653E8022F46
:1062B000D988B2EB324F4FF0000017BF92B241EADB
:1062C000014142EA014104E05A68B2EB324F08BF93
:1062D000012043E80212002AE8D1704730B4044696
:1062E00054E8000F0D4644E80053002BF8D1156028
:1062F00030BC704730B4044654E8000F40EA010552
:1063000044E80053002BF7D1156030BC704730B41F
:10631000044654E8000F00EA010544E80053002B4E
:10632000F7D1156030BC704730B4044654E8000F14
:1063300080EA010544E80053002BF7D1156030BC1A
:10634000704730B4044654E8000F00EB010544E800
:106350000053002BF7D1156030BC704730B40446B1
:1063600054E8000FA0EB010544E80053002BF7D1DF
:10637000156030BC704770B404464FF0000054E81C
:10638000006F0D68AE4207BF44E80023012044E8D7
:1063900000630E60002B1CBF0020F0E770BC70474C
:1063A00030B4044654E8000F88422CBF451A054615
:1063B00044E80053002BF5D1156030BC7047000055
:1063C0000648804706480047FEE7FEE7FEE7FEE78F
:1063D000FEE7FEE7FEE7FEE7FEE7FEE7C567020031
:1063E000016202002DE9F05F0546002092469B46BF
:1063F00088460646814640241BE0284641464746DB
:10640000224600F06BF853465A46C01A914110D309
:1064100011461846224600F016F82D1A67EB0108BF
:106420004F4622460120002100F00DF817EB00092D
:106430004E41201EA4F10104DFDC484631462A46C5
:106440004346BDE8F09F202A04DB203A00FA02F11F
:10645000002070479140C2F1200320FA03F3194352
:106460009040704700487047F800030040EA01037D
:106470009B0703D009E008C9121F08C0042AFAD2FA
:1064800003E011F8013B00F8013B521EF9D27047BE
:10649000D2B201E000F8012B491EFBD27047002266
:1064A000F6E710B513460A4604461946FFF7F0FF13
:1064B000204610BD421C10F8011B0029FBD1801A98
:1064C000704730B504460020034600E05B1C934251
:1064D00003D2E05CCD5C401BF8D030BD202A04DB49
:1064E000203A21FA02F00021704721FA02F3D0404D
:1064F000C2F120029140084319467047064C074DEF
:1065000006E0E06840F0010394E807009847103483
:10651000AC42F6D3FFF778FE3C0903005C090300A8
:1065200070B58C1810F8015B15F0070301D110F855
:10653000013B2A1106D110F8012B03E010F8016B82
:1065400001F8016B5B1EF9D12B0705D40023521E05
:106550000DD401F8013BFAE710F8013BCB1A921C6D
:1065600003E013F8015B01F8015B521EF9D5A1426B
:10657000D8D3002070BD00002DE9F04700268AB076
:10658000DFF85091B0464FF48075012437460696E7
:10659000284605F069F938B1D9F80403204203D040
:1065A000284605F057F926432D1D64007F1CADB227
:1065B000082FEDD34FF4BE74204605F055F948B1CD
:1065C000204605F047F946F0004606AA01210020C2
:1065D00005F02CF9404D16F0FF0F15D001270024CF
:1065E00037420DD009EB8401D1F81005D1F8101510
:1065F000C0F3042055F82420C1F3014102B19047B3
:106600007F00641C082CEBD3002E5FDA4FF0FF30C4
:10661000CDF8108054E0281910F8507F90F9000050
:1066200027F0C008401C3BD007A9404604F099FA67
:1066300010B34FEA9719404602F0CEF855F8207093
:106640001FB1B9F1030F03D006E0B9F1030F27D151
:1066500004A9404604F08DFA4FF0A04101EB8800F8
:10666000D0F8000706A9C0F3014A404604F079FAC1
:1066700018B1BAF1020F03D012E0BAF1030F0FD133
:10668000B9F1030F08D1BAF1020F1DD00221404623
:1066900005F0B0F8761CF6B217B149464046B84747
:1066A000641C042CB7D3002E10D06A4601210020B0
:1066B00005F0BCF806990098884207D00690049827
:1066C000002634460790A6E70321E0E70AB0BDE8BC
:1066D000F0870000006000401829002000F01F0231
:1066E000012191404009800000F1E020C0F88012B3
:1066F000704700F01F02012191404009800000F125
:10670000E020C0F80011704700F01F020121914005
:106710004009800000F1E020C0F8001270474907EE
:10672000090E002806DA00F00F0000F1E02080F8E2
:10673000141D704700F1E02080F80014704700003D
:1067400070B54FF48076304604F04AFB114CB50525
:1067500060B1304604F04BFB0120C5F808036079B6
:1067600020B9012060712168002088474FF48276AB
:10677000304604F035FB00280AD0304604F037FBE1
:106780000220C5F808032168BDE8704001200847D1
:1067900070BD0000B822002007480021C0F8401159
:1067A000C0F84411C0F84811C0F84C11C0F80011ED
:1067B000C0F8041108F0FCBC0010014008F046BC11
:1067C00005F00ABEF0B5B5480023021D0178101D82
:1067D00001254FF0805406290BD11678360708D1D1
:1067E0000678C6F30316032E06D0042E04D0052E19
:1067F00002D0062907D00EE0B4F82463A84FC6F3F0
:1068000004263E6002E01678360704D10678C6F307
:106810000316032E02D0062904D00FE0A24FA14E8A
:106820007E670EE01678360708D10678C6F30316A1
:10683000032E06D0042E04D0052E02D0062907D040
:106840000EE0D4F84462994FC6F342363E6002E04F
:106850001678360704D10678C6F30316032E02D045
:10686000062906D011E0924E376827F0807737600E
:106870000EE01678360708D10678C6F30316032E05
:1068800006D0042E04D0052E02D006290AD011E02D
:106890004FF08046C6F80C31C6F81031834E361FD3
:1068A000336002E01678360704D10678C6F3031683
:1068B000032E02D0062905D00CE07C4F0326643756
:1068C0003E600AE01678360704D10678C6F3031650
:1068D000032E02D006290DD014E0764F05263E6027
:1068E000744E78363560734E083633603F263F1D50
:1068F0003E6002E01678360704D10678C6F3031628
:10690000052E02D0062957D062E06B4E36686B4FD9
:106910003E60694E361D36683F1D3E60664E083645
:1069200036683F1D3E60644E0C3636683F1D3E6043
:10693000614E103636683F1D3E605F4E1436366835
:106940003F1D3E605C4E183636685C4F20373E6017
:10695000594E1C3636683F1D3E60574E203636680D
:106960003F1D3E60544E243636683F1D3E60524EF9
:10697000283636683F1D3E604F4E2C3636683F1D28
:106980003E604D4E303636684C4F40373E604A4E82
:10699000343636683F1D3E60474E383636683F1DF8
:1069A0003E60454E3C3636683F1D3E60424E4036A6
:1069B00036683F1D3E6002E01678360708D106783B
:1069C000C6F30316032E06D0042E04D0052E02D0E3
:1069D000062907D019E0D4F85812394A01F04F01BE
:1069E000116002E0117809070FD10078C0F303109D
:1069F000032803D0042801D0052806D131480168B6
:106A0000C90702D06FF001010160D4F830010628F7
:106A100008D1D4F83401062804D12B48016841F488
:106A20008061016022487438016841F4700101609E
:106A3000BFF34F8FBFF36F8F4FF01021D1F80002DB
:106A4000002803DBD1F80402002822DA1F4A15606F
:106A50001F480468002CFCD01524C1F800420568CA
:106A6000002DFCD0C1F8044201680029FCD013605D
:106A700001680029FCD0BFF34F8F0D48F038016842
:106A8000144A01F4E06111430160BFF34F8F00BF6E
:106A9000FDE7124910480860F0BD0000E00F00F06B
:106AA000403501400DF0ADBA00C007403C05004044
:106AB000FCED00E0105600400404001020C500402A
:106AC000E40E0040000400403C17004004E5014093
:106AD00000E401400400FA050090D003DC2300200C
:106AE0000148006800470000C022002002E008C8FA
:106AF000121F08C1002AFAD170477047002001E038
:106B000001C1121F002AFBD170470000012120287B
:106B100003DA81400548014003E0402802DA2038CA
:106B2000814009B10120704700207047FC06FFBD7D
:106B3000082806D228B1012803D0042801D001205A
:106B400070470020704710B560B159B102780B78DA
:106B50005208B2EB530F05D10622401C491CFFF727
:106B6000B0FC08B1002010BD012010BD800701D08D
:106B70000020704701207047C3688B4206D811443B
:106B80000069491E814201D80120704700207047EA
:106B900010B501220221002001F022FC08B10728D3
:106BA00010D107220221012001F01AFC08B10728A8
:106BB00008D100210A22084601F012FC08B107287A
:106BC00000D1002010BD000010B550B10A480321CB
:106BD000008801EB004009A105F036F807F012F932
:106BE00003E00321094800F0BAFC002803D0BDE807
:106BF000104000F0CBB810BD242400204572617312
:106C00006520626F6E647321000000005424002030
:106C100070B58CB015460E4600236C46C3F10F01CB
:106C2000415CE1545B1C102BF8D30D2104F11000E2
:106C3000FFF735FC0020C0F10F02315C2244401CFC
:106C400011740328F7D3684646DF0020C0F10F0116
:106C5000214491F820102954401C0328F6D30CB08D
:106C600070BD022001F0C6BA0149097900F00ABEE0
:106C70008822002070B50024064D06E068680121D6
:106C800010F8340005F092FC641C28788442F5D397
:106C9000002070BDC8220020F8B515460C460646F7
:106CA000052A01D20720F8BD05F07CFD18B905F0D2
:106CB00041FD0028F7D1124900224E600C708D6012
:106CC000C1E90422C1E906220E4D0DE006EBC40025
:106CD0002968009181788DF8011000780A4A694688
:106CE00005F0B6FC0028DED1641EE4B2EED2BDE8A9
:106CF000F84004480021054A001D00F099B8000042
:106D0000C822002070FD020041980200258C02007C
:106D100072B605F04FF800BF04F086FE0028FBD1E4
:106D2000104C0121208801EB00400FA104F08CFFE2
:106D300010480068C00700D000BE2088022101EB87
:106D400000400DA104F080FFBFF34F8F0948E438E5
:106D500001680D4A01F4E06111430160BFF34F8FF8
:106D600000BFFDE724240020466174616C20657239
:106D7000726F7200F0ED00E053797374656D2072EC
:106D800065736574000000000400FA050EB500216B
:106D90000091CDE901106A4644F20100FFF7B8FF07
:106DA0000EBD000070B502280DD1084C032508A1C6
:106DB000208805EB004004F047FF208810A105EB78
:106DC000004004F041FF012070BD00002424002099
:106DD000506F776572206D616E6167656D656E7469
:106DE0002077616E747320746F20726573657420F0
:106DF000746F20444655206D6F64652E00000000BE
:106E0000506F776572206D616E6167656D656E7438
:106E100020616C6C6F77656420746F207265736598
:106E20007420746F20444655206D6F64652E0000F9
:106E3000074B9B7823B12AB120B10068037C1BB1BA
:106E40000820704707207047417442610020704756
:106E5000E429002070B507F0FFFA104800240B2148
:106E6000047044700E4D817014206C602C706C7036
:106E7000FFF734FC07211420FFF751FC1420FFF723
:106E800038FC0848046007211120FFF748FC05483A
:106E9000001F0068A860002070BD0000E4290020E9
:106EA000E8220020081501402DE9FC47DFF8789022
:106EB00099F8023073B368B3052902D20720BDE800
:106EC000FC87436933B3437C012B25D0002704465C
:106ED0000025884616468DF80050684600F038F8C0
:106EE00001A808F0FBFBC8B1012101700F49446003
:106EF0000968C0E90218C0E904769DF8040089F821
:106F000001009DF8000000F047F81420FFF7FCFB9B
:106F10002846D4E70820D2E70F46D8E704259DF895
:106F2000000000F039F8F3E7E429002004150140DF
:106F30000649897839B130B1416921B10021017424
:106F4000022108F011B9082070470000E429002050
:106F500030B5EFF3108172B60D4A9468012324B165
:106F60000370002900D162B630BD93604FF0E0237A
:106F7000D3F88051074C25401560C3F88041D3F801
:106F8000844154605A17C3F8842100220270E8E754
:106F9000F02A0020FC06FFBD0B498A68002A11D0A8
:106FA00000280FD1EFF3108072B60B684FF0E0228B
:106FB000C2F800314B68C2F8043100228A60002810
:106FC00000D162B670470000F02A00202DE9F041A0
:106FD000064608680C46411C4FF0A0474FF00105DB
:106FE00006D005FA00F1C7F80815206804F0EEFB9A
:106FF0006068411C02D0002104F0D6FB3168A06912
:10700000C1F82405607D227D31681043C1F86C050C
:10701000D4E900123068C0F81425C0F80C15207DA2
:10702000012815D1A068411C02D0002104F0BCFB4E
:10703000E068411C05D08540C7F80855E06804F0B9
:10704000C5FBD4E902123068C0F80825C0F8101555
:10705000BDE8F0812DE9F041064608680C46411C68
:107060004FF0A0474FF0010506D005FA00F1C7F830
:107070000815206804F0B4FB6068411C02D00021B0
:1070800004F09BFB3168A069C1F82405607D217D77
:1070900032680843C2F86C05D4E900123068C0F8C1
:1070A0000C15C0F81425207D012815D1A068411CBD
:1070B00002D0002104F081FBE068411C05D085402E
:1070C000C7F80855E06804F08BFBD4E90212306879
:1070D000C0F80825C0F81015BDE8F08103F04EB9DE
:1070E0002DE9F047074600888EB0804602F03CFE4E
:1070F000824604462D4800252A460178404600F085
:10710000D9FB7879400734D501254FF6FF7603ABDC
:107110002A460721504606F059F8010004D040469F
:1071200007F0B4FB00252BE0B1463146049802F08D
:107130006FFD064648450FD004460146404602F022
:10714000FDFD4046FFF790FD30B9404607F070FB6B
:107150004046FFF789FD48B122460721504606F018
:10716000ABF8010003D0404607F090FB00254E45E8
:1071700006D0404606F00EFA10B1504602F0E0FD8F
:1071800002208DF81800ADF81A807879400701D5F3
:10719000012000E002208DF820008DF8215006A883
:1071A00001F000FF0EB0BDE8F0870000882200204B
:1071B0002DE9FC47002517880646158090F82D001C
:1071C0001446894630B13A462146484600F09CFBB9
:1071D000051E09D1B0784FF00C0A18B32088C846B4
:1071E000001DB84202D95046BDE8FC87684679DFE9
:1071F0000028F9D12088032108F8001020881921DF
:10720000401C80B2208008F800102088401C80B20A
:10721000208000EB0801BDF8000008F08DF92188FE
:1072200008442080F0780222C8B1218896F9033002
:1072300001F1030C4846BC45D5D8425421884FF093
:10724000010C491C89B2218000F801C02188491C29
:1072500089B2218009F801302088401C20807068A4
:10726000B8B1218890F9003001F1030C4846BC45C3
:10727000B9D8425421880A22491C89B2218042543B
:107280002188491C89B2218009F801302088401CDE
:107290002080308950B1CDE900474B4606220221BB
:1072A00006F1080008F032FA051E9DD1308A50B16F
:1072B000CDE900474B460722032106F1100008F0F4
:1072C00025FA051E90D1308B50B1CDE900474B46D1
:1072D0001522142106F1180008F018FA051E83D1B2
:1072E000306A30B13B462246494601F030FB051E6C
:1072F000DBD1706A30B13B462246494603F0ECF9D7
:10730000051ED2D196F82C0038B13B46224649469C
:10731000304607F061FB051EC7D1307838B13B46D7
:1073200022464946304603F05DFA051EBDD1284687
:107330005AE718B504460020ADF8000013466A4627
:10734000204600F006F8002802D0BDF800002044D6
:1073500018BD70B588B182B10024158803E0065DC0
:10736000641C3444A4B2A54203D8061976789E4220
:1073700001D08C42F3D38C4201D3002070BDA11CFC
:107380001180005D401E80B270BD80F830107047E3
:107390002DE9F0410D00044606D02CB195F87A0095
:1073A0000026012803D006E00E20BDE8F08195F804
:1073B0009800012829D0D5F8A000042825D0D5F8B8
:1073C0009C00042821D04FF00108A6702C2205F162
:1073D0007801201DFFF74AF884F83060D5F8A40042
:1073E0006063D5F8A800A0634FF6FF70A4F8A8006A
:1073F00004F19400C4F8A400C4F8AA60A4F8AE6034
:1074000084F8B060207810B104E00720CDE7FF20B9
:1074100084F8540004F155011F27C4F89410A4F80F
:10742000987004F198022846FFF7C2FE0028BCD1EC
:1074300015F13C0F0ED004F17401C4F89C10A4F8AF
:10744000A07004F1A00205F13C00FFF7B1FE002896
:10745000ABD103E0C4F89C60A4F8A06084F851802C
:10746000208BA4F8480084F83C80266484F850609F
:1074700060696064454604F13C02002104F1540057
:1074800072DF002891D125708FE710B50288102A8D
:107490001BD0112A20D0262A1DD1007A0C460128A3
:1074A00001D0022817D1A0780521401CB0FBF1F2D1
:1074B00001FB1201204600F052F800280BD0A16B0E
:1074C000002908D0BDE810400847C27B012A02D13C
:1074D0008088A1F8A80010BD0C46002184F8B210E5
:1074E0008088B4F8A8108842F5D120790028F2D11C
:1074F0000121DFE710B50C46022801D0032810D186
:10750000607800280DD000206070A178204600F03F
:1075100026F8002805D0A16B002902D0BDE8104054
:10752000084710BD10B5044690F8540074DF0120E0
:1075300084F8B200002084F8B40084F850000621DA
:10754000204601F035FF002808D1A178204600F040
:1075500006F810B1A16B01B18847002010BD2DE9DC
:10756000F05F044600780F4638B1A770002003F0A2
:1075700041FF012620B1667007E10820BDE8F09FB9
:107580000025C4F8AA50A4F8AE5084F8B050A079F1
:1075900010B1A078012806D0E07968B1A078012860
:1075A00001D0022808D1616B21B184F8B1600820B4
:1075B000884701E084F8B15004F1AB0100200A5C77
:1075C0000AB1304603E0401C0628F8D300204FF0F3
:1075D00002084FF0030B012F06D0022F0CD0032F0F
:1075E0000FD0042F15D110E0A17929B194F82410FF
:1075F00011B908B130460DE0E17911B108B140464A
:1076000008E0207A08B1584604E0607A08B1042006
:1076100000E02846A070616B41B1032801D0042826
:1076200004D1607910B194F8B200A0B184F8B350DD
:1076300004F13C0018210746FEF731FF04F12C004D
:1076400084F83C60814606F0E1F858B194F82C00CB
:1076500084F8510008E084F8B45084F8B36007203F
:107660008847E5E784F8516094F8240050B1484613
:1076700006F0CCF820B194F8280084F8520001E01C
:1076800084F8526084F85050A27804F1AA0104F101
:1076900094094FF0060A052A60D2DFE802F0780369
:1076A0000F223F0084F83160C4F8A450C4E91015DB
:1076B00084F83C808020A4F8480051E084F83180B0
:1076C00094F82420384612B10722027001E080F8B5
:1076D00000B0228A8281C4F8A4504160E168B96098
:1076E0003EE06069B860208BB88194F824003D4684
:1076F00010B184F83CA001E084F83C60204607F01B
:10770000C9FF40B185F814800421204601F050FEE5
:1077100020BB05211EE084F831B01DE0E069B860AF
:10772000208CB88194F824003D4610B184F83CA028
:1077300001E084F83C60204607F0ACFF48B185F8D2
:1077400014800421204601F033FE38B984F831A0BA
:1077500002E0042184F83110C4F8A490A07878B134
:107760003A4604F15400D4F8A41072DF00287FF4E4
:1077700005AF94F8301094F8540073DF0028F6D168
:10778000616B11B194F8310088470020F6E684F867
:107790003150F5E770B5040012D001461C221448A0
:1077A000FEF764FE1248134D0560206850B17ADF81
:1077B000002806D12068016829604068686005E0FB
:1077C0000E2070BD0B487BDF0028FAD108484FF629
:1077D000FF711438084A20F8041B05493439016048
:1077E0000021FFF725FB0028EBD0032070BD00002F
:1077F000AC250020482200202DF6020010B50446DA
:1078000000F078F8002805D02146BDE81040024875
:1078100003F00BB910BD0000D825002070B5154647
:107820000E46044607F042FF002809D0054800EB49
:10783000840080692A463146BDE8704001F0F6BDFB
:1078400070BD0000C825002070B50546002400F07A
:1078500051F838B12946044803F0E7F808B102248A
:1078600000E00124204670BDD425002010B5182169
:10787000034803F0B5F8182800D0C0B210BD0000CE
:10788000C825002070B505460C46084607F00EFFD7
:1078900060B1284600F02EF840B10548294600EBBB
:1078A0008400BDE87040183003F0BFB8002070BD00
:1078B000C825002070B5054614460E46084607F058
:1078C000F5FE002812D0284600F014F800280DD04C
:1078D0000748294600EB860018301CB1BDE870400F
:1078E00003F0AEB8BDE8704003F05FB870BD0000B3
:1078F000C8250020142801D3002070470146014804
:1079000003F093B8CC2500207CB5054608880C46CA
:107910000930904201D90C207CBD68466DDF0028FB
:10792000FAD121880820685420881B21401C80B28D
:10793000208029542088401C80B220802844DDF813
:1079400001100160BDF8051081802088801D80B283
:1079500020809DF80010490800D00121295420887A
:10796000401C208000207CBD10B503F049FA00289F
:1079700009D105484FF0020C00DF002803D1BDE813
:10798000104003F0A1BA10BDB828002020B103496F
:107990000860034806F06ABA0E207047A82200204B
:1079A0003DDA020010B54FF0FF3100203DDF002826
:1079B0000BD1B1213CDF002807D1044841690120E7
:1079C0008847022004F01AFB002010BD9C280020EC
:1079D00070B50E4C2068416900208847206813214B
:1079E000808876DF050008D009480121008801EB76
:1079F000004008A104F028F905E005F0B3FE216875
:107A0000086101F077FF284670BD0000A822002021
:107A1000242400204661696C656420746F206469C9
:107A200073636F6E6E6563742047415020636F6EA1
:107A30006E656374696F6E0030B58FB005461C21AA
:107A400001A8FEF72CFD0024142109A80894FEF7D4
:107A500026FD9DF82000009420F00F00401C20F02F
:107A6000F00010308DF820009DF82100029420F0E5
:107A70000F00401C20F0F00020308DF821009DF810
:107A80002200049420F00600801C8DF822009DF84E
:107A9000040009AA40F028008DF8040008A8CDE9E8
:107AA0000540079428788DF83A000420ADF8380096
:107AB0009DF80000ADF82C4020F00F00401C20F095
:107AC000F00010308DF800009DF80100ADF82E4058
:107AD00020F00F00401C20F0F00020308DF8010055
:107AE0009DF802000D9420F00600801C20F0080094
:107AF00040F011008DF802000EA809901720CDF873
:107B000028D0ADF830006888AB1D01A9AADF0FB0FE
:107B100030BD000010B5164C86B01ECC8DE81E009E
:107B200020B3144C4FF6FF71A18000686061002003
:107B3000607620762046FFF729FF002814D1012027
:107B40008DF812004FF65960ADF81000A21C04A980
:107B50000120A8DF002807D12146684662DF0028FF
:107B600002D12046FFF768FF06B010BD0E20FBE7EC
:107B700054FD02009C28002010B500280FD0018879
:107B8000204C502926D00BDC10291DD0112906D1FC
:107B9000A1888088814202D14FF6FF70A08010BD7D
:107BA000512913D05329FAD1C088E1888842F6D1EF
:107BB000607E0028F3D0FFF70BFF0028EFD061694B
:107BC000BDE81040022008478088E7E7BDE8104084
:107BD00005F0FCB830F8061F62899142DFD1418977
:107BE0000229DCD10C3000F0BDFA074920760322CF
:107BF0000988BDE8104002EB0143024603A1184684
:107C000004F026B89C2800202424002052656365D7
:107C10006976656420696E6469636174696F6E205A
:107C200073746174652025640000000070B505461A
:107C3000007B0424012810D00224287B214600F078
:107C400051F80C4C18B1206841690320884720681E
:107C50004169BDE870400220084701F05FF8002844
:107C600007D0112803D00F28E7D10724E5E7062421
:107C7000E3E770BDA822002070B5184900250A6806
:107C8000002A2AD04A68002A27D0012608319047C6
:107C9000082822D0124C0028206810D0457685761E
:107CA0000621012000F01EF818B120684169032068
:107CB000884720684169BDE8704002200847467641
:107CC00085760121084600F00DF8002805D02068CF
:107CD0004169032088472068457670BDB828002098
:107CE000A822002086B00323ADF8003020238DF8B1
:107CF00014308DF8150000220E48019202928DF882
:107D00001610C188ADF8041002218DF8061005A9DF
:107D10000491ADF80820CDF80CD0808801A9AEDF21
:107D2000002804D1BDF80010032900D00C2006B0B3
:107D3000704700009C2800200F4A0321128801EBA5
:107D4000024268B101280ED00B4A01210228128894
:107D500001EB02420AD0032810460AD007A109E02D
:107D6000104610A106E010461AA103E0104622A119
:107D700000E030A103F068BF24240020556E6B6E34
:107D80006F776E206576656E742066726F6D206207
:107D90006C655F6466755F627574746F6E6C657335
:107DA000732E0000446576696365206973207072E4
:107DB00065706172696E6720746F20656E7465729C
:107DC00020626F6F746C6F61646572206D6F6465A3
:107DD0002E0000004465766963652077696C6C202D
:107DE000656E74657220626F6F746C6F616465722A
:107DF000206D6F64652E0000526571756573742087
:107E0000746F20656E74657220626F6F746C6F6141
:107E1000646572206D6F6465206661696C656420BD
:107E20006173796E6368726F6E656F75736C792EAE
:107E3000000000005265717565737420746F2073C3
:107E4000656E64206120726573706F6E7365207457
:107E50006F20636C69656E74206661696C65642E61
:107E60000000000038B50446008821281CD013DC2F
:107E7000102822D1072000F0D5FA08B1FEF786FFBE
:107E80001048A1880180104802F032FF002814D069
:107E9000BDE83840FEF77ABF3B280FD056280CD1FA
:107EA000A088132176DFF1E700200090A0886946C2
:107EB0008FDF002801D0FEF769FF38BDA0881321AD
:107EC00076DFE3E7282200204824002010B51A4C72
:107ED0000188606810290ED011292BD1401E6060E6
:107EE00028D1FEF755FE002824D02168002921D092
:107EF000BDE810400847D0B900210122084600F033
:107F00006FFA08B107280FD107220221012000F0E3
:107F100067FA08B1072807D104220221002000F0E7
:107F20005FFA20B1072802D0216801B18847606854
:107F3000401C606010BD0000402200202DE9F04789
:107F400001883B4E40F2F3194FF6FF7510291BD004
:107F500011293ED0122954D0502946D1C188F28926
:107F6000841D914241D1618902293ED186883046E3
:107F700001F0A6FF050038D004F10C0000F0F6F87F
:107F8000A8B3294630464EE0C17B878804460129C4
:107F90002BD1A846284601F093FF050017D02F806B
:107FA00000202872234843464A460168C5F80A1053
:107FB0004068C5F80E0004F1100105F10A0002F056
:107FC0004BF86872F08900280FD129462AE0042076
:107FD00013E0808801F074FF040006D06068FEF7AB
:107FE000A7FF08B106F036FC2580BDE8F087FFE763
:107FF0006868FEF79DFF0028F7D0BDE8F04706F05F
:1080000029BC87880646384601F05AFF0400ECD0A8
:108010002B464A4606F1080104F10A0002F01CF85A
:10802000607221463846BDE8F04700F0D7BC00003A
:10803000AC250020482200202DE9F04F0746858816
:1080400002883D48012197B08346102A09D0112AA1
:1080500049D01A2A6CD1387AB1EB101F45D20122CF
:1080600044E0354C083CA068C0430B9061680BA805
:1080700002F0FFFC0B990CA800F04AFC2C220CA982
:108080006846FEF7F3F90026E946A04610E000BF77
:1080900009EB46005FF00004B0F804A008EB840090
:1080A0005146001D02F081FC641C1D2CF6D3761C89
:1080B0000098B042ECD8142D05D317B00420BDE8C9
:1080C000F04FFEF763BE2946584602F0B9FC294638
:1080D00008F1040002F0B4FCF87B012828D016480F
:1080E0002946001D15E029461AE000220221B1EBC5
:1080F000101F01D2012600E000260F49083901F1C6
:108100001000041D294682B102F09AFC36B12946BE
:10811000204617B0BDE8F04F02F092BC2946204639
:1081200017B0BDE8F04F02F040BC02F03EFCF5E7AE
:1081300017B0BDE8F08F0000D025002010B5044630
:108140000748007800280AD0204601F0E7FC2046C6
:1081500006F0DAFC2046BDE8104001F073BA10BD0D
:10816000782200200078C0F340007047007800F0CB
:10817000010070470149085C704700000CFC0200D8
:108180000649095C4FF0A040D0F81005C84010F037
:10819000010000D0012080F0010070470CFC0200BB
:1081A0002DE9FC410646C0074FF000050ED0104FE8
:1081B00000240122385D009500231146019503F04B
:1081C00099FA641C042CF4D300F046F8B0070DD5DE
:1081D000074E0024361D0022305D03230095114612
:1081E000019503F087FA641C042CF4D3BDE8FC81EC
:1081F00008FC020007490B5C4FF0A041D1F80425B0
:108200000120984020EA0203C1F808351040C1F867
:108210000C05704708FC02000249085C012103F0CC
:10822000FABA000008FC02000249085C002103F0D1
:10823000F2BA000008FC02000649095C4FF0A040B9
:10824000D0F80405C84010F0010000D0012080F0F3
:108250000100704708FC020010B500242046FFF71B
:10826000DBFF641C042CF9D310BD10B5002420469C
:10827000FFF7DAFF641C042CF9D310BD10B50246D9
:10828000064B4FF0FF3000215C5C944201D1084660
:1082900010BD491C0429F7D310BD00000CFC0200DE
:1082A00070B50C4E0C004FF0000530600BD0012073
:1082B00000F06AF808B1022004E0002000F064F841
:1082C00000B10B202070706810B9FEF761FC054604
:1082D000284670BD4022002010B5002000F0D4F9DF
:1082E00008B1062806D1012000F0CEF908B1062811
:1082F00000D1002010BD00002DE9F0470D46814659
:10830000FFF7BCFF0446042836D2DFF874801B4810
:108310001C4EA8F10C0725B3012D0ED0022D2BD138
:1083200004EB440030444578002D25D0B96800297D
:1083300022D02846BDE8F047084704EB4401755CAD
:108340000E44717849B10E4A4FF40041093A8068F1
:10835000FEF7AAFD08B987F80390B17808F8041071
:10836000E2E78068FEF7E4FD04EB4401314418F8CD
:1083700004008D78A842D7D0BDE8F08710FC020039
:108380003C2200204C250020042801D2FFF7F8BE33
:10839000002070470146104810B50088042907D016
:1083A00007290ED00A2915D1BDE8104006F096BB6A
:1083B000132176DF0CE000280CD0BDE81040FEF75A
:1083C000E5BCA0F57F41FF3904D10448FFF7AAF8C6
:1083D0000828F0D110BD00002822002054240020DD
:1083E00070B50023042810D20D4D00EB4004012A83
:1083F00002D101290CD00022094E00EB400030448C
:1084000061B1012906D0022906D00723184670BDA4
:108410000E30C2B22A55F9E74270F7E78270F5E7ED
:108420004C250020044A014600201279D20702D0D0
:10843000084600F04DB870473022002070B506465F
:108440001E480024C0E90161B00720D500250122A3
:1084500011462846FFF7C4FF6D1C0446042D02D2C6
:10846000002CF4D013E094B940F266620421144861
:10847000FEF712FC04000AD1FEF7FCFB040006D153
:108480000F48104A0021001FFEF7D2FC0446F007F7
:1084900012D00120FFF784FE74B909480A4A00216E
:1084A0000C38FEF7C5FC040006D10548074A012137
:1084B0000838FEF7BDFC0446204670BD302200207F
:1084C0001CFC020055870200EDA00200636C020054
:1084D0002DE9F05F6A4C054600266078B34618B176
:1084E00084F801B001F0EAFD664F4FF47A694FF469
:1084F000C87A4FF00108182D62D2DFE805F0AC0C05
:108500000C31404D62676B746B74BE7D7D7D7D7DEB
:10851000ACAFB2B5BEBE0020FFF78EFE00284FF014
:10852000000008D0FFF778FE022D02D14FF4E16081
:1085300008E0484606E0FFF777FE022D01D1C8208B
:1085400000E05046410CC0034FF4FA72801841F12C
:108550000001257052000023FDF744FF01462AE088
:108560000020FFF769FE00284FF0000004D0FFF75D
:1085700053FE4FF44870E5E7FFF756FEDFE70020B3
:10858000FFF75AFE00284FF0000002D0FFF744FE2C
:10859000CFE7FFF749FED4E70020FFF74DFE0028A4
:1085A0004FF0000002D0FFF737FE01E0FFF73CFE7E
:1085B000257041F69A1100223868FEF775FC0646D0
:1085C00046E00020FFF716FE257008E0002051E08D
:1085D00025703DE084F801800120FFF70BFE0022AA
:1085E00040F6CD41E8E784F801800120FFF702FE64
:1085F00000224FF48041DFE77868FEF799FC0646D9
:10860000D5F1110000D02EB10220FFF705FE84F84D
:1086100002B01DE0012816D980B2C8214843C11715
:10862000C90341EA5041C0034FF4FA72801841F186
:10863000000152000023FDF7D5FE014600227868B4
:10864000FEF732FC06460220FFF7EEFD84F80280BA
:108650003046BDE8F09F01F031FDB9E701F02EFD95
:10866000B4E701F02BFD04E001F028FD0020FFF746
:10867000DBFD0120FFF7D8FDAAE7FFF7F6FDA7E72E
:108680003022002010FC0200012107F0A6B80000F3
:108690002DE9F8430546861C00208DF80000904621
:1086A0000F464FF001096846FEF752FC1B4C20684C
:1086B0003860D4E90001401AA16804F21C47081A86
:1086C0000EE00121384602F0CEF901F0ADFE014680
:1086D000384602F0C8F9D4E90001401AA168081A26
:1086E000401C8642EDD8B8F1000F03D0052065F399
:1086F000891002E0062065F39F50A26821681140AE
:1087000004EB8101C8602068304420609DF80000BF
:10871000FEF742FC4846BDE8F8830000A82D002083
:1087200030B482680468531C8360A154D0E90112FC
:108730008A4202D330BC02F08ABC30BC70470000D1
:10874000034803C8814201D10120704700207047CF
:10875000A82D002000780221FFF7CEBD032805D107
:108760000349A9200860002003F048BC70470000BE
:108770002005004005494FF0FF32082841F820202D
:1087800002D3084480F848207047000018290020D0
:10879000F0B54FF0FF3512B10023082601E00823A1
:1087A0000C260C4C05E000BF54F823707F1C04D04D
:1087B0005B1CB342F8D32846F0BD26185DB286F89C
:1087C000305044F82310002AF5D1E11881F8480010
:1087D000F1E70000182900200249084490F9300010
:1087E000704700001829002070B504464FF6FF7549
:1087F0000A462846AC4208D14FF480742146104600
:1088000005F07CF9A04209D070BDFF2CFCD82146B0
:10881000104605F066F908B1204670BD284670BDC7
:1088200070B5084C050009D010342168002907D024
:1088300008682060496828468847F6E70834F4E766
:1088400070BD000004290020054A012120B1012843
:1088500005D19170FFF7E4BF51700020FAE770472F
:10886000042900202DE9F05F26484168F1B3DFF8C4
:1088700098B00E688146DBF8004087688078E11B7D
:1088800021F07F45ED1CB0B9DFF880804FF48030D7
:10889000C8F84403C8F804031120FDF71FFF112096
:1088A000FDF727FF4FF0010AC8F800A02F2003F0C2
:1088B00075FE89F802A0B54200D23546124BE81980
:1088C0003C3320F07F401860DBF800105A46091B4B
:1088D00021F07F41001B20F07F40C91C81420FD94D
:1088E000106818602F2003F059FE00E004E0BDE896
:1088F000F05F1120FDF708BFBDE8F05F05F0ACBDEB
:10890000BDE8F09FE822002004150140001001405E
:1089100073B58CB00646002000900D9880B10024FD
:108920006D4621460DA802F080F830B1009805EBA5
:10893000400084800098401C0090641C142CF0D3EC
:108940002C2269463046FDF791FD0EB070BD2DE931
:10895000F04117880646B81D14460D46984202D9C4
:108960000C20BDE8F0813188072206290AD34FF494
:10897000486C4FF6FF73614501D9994202D1708866
:10898000062801D21046ECE7604501D99842F9D19A
:10899000994203D0984201D08142F3D80520E8558E
:1089A00020881221401C80B2208029542088401C3D
:1089B00080B220804119308806F0BEFD218808442D
:1089C00080B220804119708806F0B6FD21880844E5
:1089D00020800020C5E7FEF7D9B9000038B54A7AF3
:1089E0000F4B62B100220A725969002906D0012298
:1089F0008DF80020ADF802006846884738BD0A7A35
:108A000062B19B684C68024619462046FEF74CFA54
:108A10000028F3D0BDE8384005F01CBF5B68F1E7E3
:108A2000AC250020F0B585B016460F4604461D461D
:108A300014220B496846FDF719FD0A488DF80870A5
:108A4000ADF80240ADF80A608DF80C5001780022B4
:108A50002046FEF72FFF684600F0A4FA05B0F0BDEF
:108A600028FD020088220020F0B587B007460020CC
:108A70000490ADF810100590ADF81210019002901E
:108A800001AA04A9384690DF060022D003F02CFD8D
:108A9000114C0346012520883A4605EB00400F495A
:108AA00003F0DDF8BDF8042012B9BDF8060038B1B6
:108AB0002088BDF8063005EB004009A103F0CFF88F
:108AC000BDF808202AB12088154905EB004003F0C5
:108AD000BFF807B03046F0BDF4230020FC000300CF
:108AE00054686520726571756573746564205458A7
:108AF0002F5258207061636B6574206C656E6774CB
:108B00006820697320746F6F206C6F6E67206279C4
:108B10002025752F2575206F63746574732E0000F2
:108B20004801030030B5044685B000211B4804F01D
:108B3000D8FF00282FD00025204600F01EFF68B186
:108B4000112812D086281BD0A0F54051023903D03D
:108B50000146204605F086FE294607E005B0294675
:108B60002046BDE8304001F03DBC0121204601F027
:108B700039FC05B00021BDE83040084804F0E5BFED
:108B8000142207496846FDF771FCADF802406846BB
:108B900000F0E4F9E0E705B030BD0000512200200C
:108BA00050FC02007FB50C4610B1012004B070BD2E
:108BB0002079002638B141F61D5501281BD0022826
:108BC00026D00F20F2E70220207102960396E0687B
:108BD0000190694601A805F063FB50B102988188B5
:108BE000E18000882081BDF80010029805F0D6FBD6
:108BF000DCE70A20DAE70A4B6A460021A01D05F0EF
:108C00000BFB38B1064918398E61CE610A28CDD1E7
:108C10002846CBE702488188019805F0BFFBF5E7BD
:108C2000282300202DE9F0470025DFF88C803CE068
:108C30006068002100EBC506012032789146FDF7FF
:108C400002FCD4E9062300EA020701EA030C57EA12
:108C50000C0728D082438B434846C4E9062303F01F
:108C60005FFD32788246914601200021FDF7EBFB43
:108C7000D4E9042300EA020401EA03074A46504605
:108C80000021FDF7E0FB44404F403C430BD170789E
:108C9000012801D0012100E00021726881EA0A0167
:108CA0000AB1484690476D1CEDB298F80000444662
:108CB0008542BDD3BDE8F087C822002010B5002151
:108CC000024801F0EBFE80F3100010BDC43100201B
:108CD0000E4910B50A784C780023A24212D0521CDB
:108CE000D2B20A70022A00D10B70084A0B780C32FB
:108CF00052F8232002608868104420F07F4088608A
:108D0000012010BD0360002010BD0000E8220020FB
:108D100013460A460021FFF785BE000070B5174DC7
:108D20000321288801EB004015A102F08DFF1E4EA3
:108D30003068807E28B1BDE8704006210120FEF732
:108D4000D1BF05F04FFB002816D11848A0F10C0147
:108D50000A68011F904704004FF0010002D00F2C59
:108D600003D008E03168887605E0298800EB0140EF
:108D70000F4902F069FF204670BD00002424002046
:108D800057726974696E67207065657220646174DA
:108D90006120746F2074686520626F6F746C6F61FE
:108DA0006465722E2E2E0000A8220020C428002008
:108DB000A00103002DE9F843104D0F4680461E46E2
:108DC00091466946286801F0C4FD040014D01C21B6
:108DD000FDF765FB01202071C4F81490380BC4F82E
:108DE0000080C4E902606946286801F0D3FD05F0FF
:108DF000A7F90020BDE8F8830420FBE710FE02007D
:108E000010B503780022072B06D2DFE803F0050433
:108E10000610202930000A7010BD01230B70038951
:108E20008B818388CB81C06888600A7410BD022260
:108E30000A7002898A818288CA81C2688A60807DBC
:108E4000062802D00020087410BD0120FBE7032291
:108E50000A70C2888A810289CA81C068886010BD90
:108E600004230B70C0888881CA818A6010BD0520E8
:108E7000087010BD70B5064D0646002455F8241044
:108E800009B130468847641C042CF7D370BD00003C
:108E9000082B002030B50446006887B00D46806876
:108EA00000281FD018216846FDF7F9FA0195A0683F
:108EB0000590207910B1012810D107E001208DF82C
:108EC000000020690290E068039005E002208DF820
:108ED0000000E068000302906069049020688168E7
:108EE0006846884707B030BD70B586B015460C009F
:108EF000064619D0112C17D0082C15D0142168461D
:108F0000FDF7CDFAADF80260304600F02DFFADF868
:108F100004000D2C0AD0862C1CD007208DF80000F0
:108F20000294684600F04CF806B070BD03208DF83E
:108F3000000025B12878C00701D0012000E0022000
:108F40008DF8080000208DF80C0041F20110ADF8FA
:108F50000A00E6E706208DF80000E2E710B50446B7
:108F6000408800F001FFA080024801682046BDE86B
:108F700010400847582200202DE9F0410746002400
:108F8000064E074D05E000BF56F8241038468847C6
:108F9000641CE8788442F7DBBDE8F08150280020AB
:108FA0007822002010B50446408800F0DDFEA08045
:108FB000024801682046BDE810400847FCFC02005A
:108FC000014909680847000050FD020070B586B0ED
:108FD000044614216846FDF762FAA0890125A0F530
:108FE0004040ADF8040020782A4E062833D2DFE84E
:108FF00000F0320303032C48A08900F0BDF930B91A
:10900000E08943F6FE71A0F54040884223D8A07B5A
:109010008DF80800207803280FD000208DF8090073
:10902000A0680390606850B109208DF80000606866
:109030000490684604F088F90DE00120EEE708206E
:109040008DF800008DF81050F3E7A08900F094F936
:1090500008B1E08930B17078002801D004F0A4FA9A
:1090600006B070BD606820B10B208DF800007570EF
:10907000DFE70A208DF80000BDF8040004F01EFBB5
:10908000F5E713208DF800004FF6FF70ADF80400EF
:10909000CFE700006822002038B504460E4800786B
:1090A000A8B1A4F57F40FF380FD0684604F07AFFDE
:1090B00078B10521017001210171C480684604F076
:1090C0007FFF05F02FF8002038BD042038BD0220B6
:1090D00038BD082038BD0000302300200C4808B5FA
:1090E000007888B1684604F05DFF78B10621017010
:1090F000684604F065FF0748017809B10121017352
:1091000005F010F8002008BD022008BD082008BDA9
:1091100030230020CC2B0020F0B587B01421684606
:10912000FDF7BDF92B4C207818B16846FFF7A2FE79
:109130004EE0201D01F094FCB8BB4FF010204169B7
:109140000004026940694B1C01D100FB02F1224876
:1091500000220161A1F54051C160204902F006F9E9
:10916000002820D11F481C238C221D49006801F0D3
:10917000DDFB03F0D9FE051E14D0022812D0002713
:109180000126062D12D005A804F00CFF88B1067048
:109190000C2D18D2DFE805F0170F170F171617164A
:1091A000171113110B2007B0F0BD11E02670676096
:1091B000BBE70820F7E7077105E0032100E0022183
:1091C000017100E0067105A804F0FAFE04F0AAFFA0
:1091D0000020E8E730230020E023002020FE0200EA
:1091E000182B002088FD020038B5040014D0694611
:1091F00005F056F8A0B1BDF8000000EB8001094869
:1092000000EB8100C16849B1A17A39B1C168491E3A
:10921000C1600020A07238BD052038BD062038BDD1
:109220000A2038BDA42B00201FB501A9684604F010
:10923000F3FF04B010BD07B513460A466946002087
:1092400004F0EAFF0EBD07B513460A460021684642
:1092500004F0E2FF0EBD20B119B1006808600020E3
:109260007047052070470000F8B50D46040018D07F
:10927000BDB1694605F014F8A8B1BDF800000B496E
:1092800000EB800001EB800001210C30666801F0EA
:10929000EAFB2E6060680C3068600120A07200203C
:1092A000F8BD0520F8BD0A20F8BD0000A42B002061
:1092B00018B10323002206F07FBB0520704702236C
:1092C000002206F079BB12B1022306F075BB05201F
:1092D00070470000084910B50A69042A0AD0074AF5
:1092E000096942F8210004480121103001F0BBFB5C
:1092F000002010BD0C2010BD10230020082B0020E2
:1093000038B5044609480D46007858B164B169463D
:10931000284606F04BFC002803D1BDF80010218040
:10932000658038BD022038BD052038BD30230020BF
:1093300010B504460E48007898B1A4B121880229DE
:1093400013D80C4A01EB810002EB8002608852893D
:10935000C31C934209D806F01DFC002020806080C9
:1093600010BD022010BD052010BD042010BD00005E
:1093700030230020A42B002043F6FE71A0F54040CE
:10938000884201D8012070470020704710B504467C
:109390000078182802D1FEF769FA207010BD10B5C8
:1093A00004460078182802D1FEF760FA207010BD3C
:1093B00070B50D460446B0F89810D0F8940001221C
:1093C000FDF7B7FF00B1057004F13C0204F1940110
:1093D00004F1540072DF70BD70B5134600220646DA
:1093E0001546862902D0112902D002E0012200E0B0
:1093F00001250D4C73B1A179FEF75CFA2A4661791B
:109400003046FEF757FA0022A1783046FEF752FAAE
:10941000002203E0A178FEF74DFA2A466178304633
:10942000BDE87040FEF746BA90220020F7B5174617
:109430000E0011D00098002560B100242146684636
:1094400001F0F3FA18B1A0B23946B0476D1C641CA4
:10945000142CF3D32846FEBD0020FEBD406804F066
:10946000C1BD000070B508B1012070BD194C0025C8
:10947000207B08B1257301E000F0A0F820780828CF
:1094800026D2DFE800F02504080C10251420BDE8E2
:10949000704000F021B8BDE8704000F07DB8BDE834
:1094A000704000F05FB8BDE8704000F03BB86088E5
:1094B000084900EB8000283901EB80004068BDE8D6
:1094C000704003F011BD6560BDE8704003F01ABD47
:1094D0000F2070BDCC2B00201149F0B48A1C002055
:1094E0000346A1F128050C18A67A4EB1A37200EB31
:1094F000800405EB8404E66816B9247C012C0AD0AC
:10950000401C80B20228EED30B704B804B60F0BC45
:1095100041F61D5070471080F0BC00F03DB80000CF
:10952000CC2B00200C48418801EB8102A0F12801DE
:1095300001EB8201CA6852B105210170074802217E
:109540008180016800230122054801F079BE0422D0
:1095500002704968F6E70000CC2B00203823002079
:10956000E023002038B50A49084803240B68426804
:10957000898803EB810153880470DB1C00201B04E5
:1095800000909B0B034801F0CBFF38BDCC2B002093
:1095900038230020E0230020074910B54888091D22
:1095A00004F0CEFE18B1BDE81040FFF7DBBFBDE808
:1095B0001040FFF7B7BF0000CC2B0020F0B51F48CC
:1095C0001F490125067802248B88A0F12802082E65
:1095D00019D2DFE806F00418181B222F2F17018973
:1095E000491C01810021418080F80C1001EB8103AE
:1095F00012F8233043B100234418491C89B2A372E6
:109600000229F3D30570F0BD0123F5E742685288C3
:10961000D21C1A448A800470F0BD46880D6806EB9F
:10962000860602EB860256680E60556013818C80B8
:10963000062100E007210170F0BD0000CC2B0020C6
:109640003823002030B501888488224D85B0502908
:1096500024D0522902D0542931D103E0204600F011
:109660008DFE2CE014221C496846FCF7FFFEADF885
:109670000240204600F078FBADF8040000F022F92B
:10968000002269792046FEF715F900222979204643
:10969000FEF710F96846FFF761FC10E0017B012935
:1096A0000DD1817A01290AD10089A0F5245102390E
:1096B00005D10121204600F095FE05F0ADFF002206
:1096C0000649E878FEF7AAF805B0BDE8304005F095
:1096D00011B900005022002078FC0200DD70020069
:1096E00010B50446007800280FD1608800F046FECF
:1096F000608800F08FF9002807D0044960880122B3
:109700000979BDE81040FEF7D5B810BD5022002001
:1097100010B5124C00202070FEF7A8F8A070FEF7DC
:10972000A5F8E070FEF7A2F82071FEF79FF86071CF
:10973000A17818290FD0E17818290CD0217918299F
:1097400009D0182807D00121601C04F0C3F90120BA
:109750002070002010BD032010BD0000502200200A
:109760007CB50446007808282FD1607A38BB207A6F
:109770004FF6FF7501280DD0072802D0082824D104
:109780001EE0A08800F02EFAA8421ED0012100F0B1
:1097900029FE1AE0A0886A46012103F0EDFC70B9A9
:1097A0000198007858B1A08800F01CFAA8420CD0AB
:1097B000084901220979FEF77DF805F09BF804E0DD
:1097C00004480021401C04F0C0F9BDE87C4005F0CD
:1097D00023BF00005022002010B504460A484178FB
:1097E0002046FEF74FF868B10848002101EB41021E
:1097F00000EB82025288A24201D1C8B210BD491CBE
:109800001429F3D3FF2010BD62220020402600203F
:1098100070B5094D094E002404EB440005EB8000AF
:1098200071784088FEF72EF820B1641C142CF3D315
:10983000FF2070BDE0B270BD4026002062220020F3
:109840002DE9F0418046024601200021FCF7FBFD96
:109850001A4F05460E467868FDF76AFB00280CD1C2
:10986000174CD4E9062110462A4001EA06031A43A0
:1098700005D0A843B143C4E90601BDE8F0814046E4
:1098800002F04EFF30B1D4E9040128433143C4E96A
:10989000040105E0D4E90410A943B043C4E904106D
:1098A000D4E9060128433143C4E90601A168786878
:1098B000BDE8F0410022FDF7F7BA000070FD02009C
:1098C000C82200201CB5054AD2E90212CDE90012D7
:1098D0000022694603F075FC1CBD000090FC0200EC
:1098E00003484FF6FF71818001210170002070470D
:1098F0005C22002010B54FF6FF7003F0F7FB034920
:109900008880BDE8104004F0FFBF00005C2200200A
:109910002DE9FC41804600F027FA002403250127A9
:10992000A0F57F412646FF3908D06A46082103F09A
:1099300023FC18B90198841D8688056832462B4699
:1099400021464046B1DF042804D0082804D00B2863
:1099500008D002E0112000E00020002F00D10B20F1
:10996000BDE8FC810027A80701D50125E6E73443BF
:10997000F5D0002426460325E0E72DE9FC4180468A
:1099800000F0F2F90646A0F57F40FF380ED0012521
:109990002A466D1C0027ADB26B460821304603F005
:1099A00015FC040006D0072C25D025E043F2020068
:1099B000BDE8FC81019903230A1D0B604046891D07
:1099C000B2DF040004D00C2C09D0052C09D009E02A
:1099D00032460821104603F06FFC04460CE00127D4
:1099E00000E000240821304603F052FC00B10324BB
:1099F000002FCDD100E00C242046D9E70448808810
:109A0000A0F57F41FF3901D004F07EBF7047000010
:109A10005C2200200EB502A9019100F0A5F96A466A
:109A2000012103F0A9FB08B100200EBD01980078C8
:109A30000EBD00002DE9F04107464FF6FF760A48BB
:109A4000B3DF10B10320BDE8F081074C43F20305FA
:109A5000A41E324661883846AFDFA842F3D1608841
:109A6000401C6080F5E700005E220020428800EB89
:109A700082020C328A4201D9022070478188A1F506
:109A80007F42FF3A03D0008808B1002070470120D0
:109A90007047884204D20068401C01D00120704702
:109AA000002070473EB5027802230C46B3EB520FFC
:109AB00017D1B0F80110ADF80010C1788DF8021080
:109AC0008188ADF8041080798DF8060002AA01A9FA
:109AD0002046FDF79DF8032202A96846FCF7F1FC39
:109AE00008B100203EBD01203EBD000010B50C466F
:109AF000FFF772FEFF280CD0074900EB400001EB96
:109B00008000416821600189A180807AA0710020D5
:109B100010BD052010BD00004026002070B5018852
:109B200090B0102959D1011D2C226846FCF79EFCEB
:109B30009DF804004FF6FF76032134466D46B1EBE5
:109B4000500F2AD003F06EFC9DF8040040080ED0A0
:109B500001280CD0022820D118E00D99281D1131C0
:109B6000FCF7F1FF18B100BFBDF82C4015E00CAABE
:109B70000BA9072003F02AFC0028EED10DE00D9977
:109B8000281D491CFFF78EFF0028EDD10CAA0BA958
:109B9000072003F01BFC0028F1D1BDF80000291DAF
:109BA00000F06EFEB44218D0BDF80000214600F06F
:109BB000C5F8BDF80000ADF82E000020ADF830402B
:109BC000074E8DF82C000BAD044600BF56F824104C
:109BD00028468847641C022CF8D310B070BD0000E2
:109BE000A4FC0200094A002101EB410332F82330B2
:109BF000834205D101EB410002EB800040887047B1
:109C0000491C1429F0D34FF6FF70704740260020FE
:109C10003EB50C46054603F005FC0BE0BDF8000020
:109C2000A04207D02846029900F02EF810B1BDF8E6
:109C300000003EBD01AA6946072003F0C7FB0028CB
:109C4000ECD14FF6FF703EBD10B50D4C18200D4AFB
:109C5000607000204FF6FF7100EB400302EB8303BE
:109C6000401C59801428F7D3FDF700FE60701828B7
:109C700003D001202070002010BD032010BD000083
:109C800062220020402600202DE9F0410C460546C6
:109C900000F1110701F111061022491C401CFCF7CC
:109CA00010FC48B9681C00F0F9F928B1601C00F0FC
:109CB000F5F908B1012400E0002431463846FCF7EC
:109CC00042FF3B780222B2EB530F0CD00321B1EBE1
:109CD000530F08D03378B2EB530F04D0B1EB530FCE
:109CE00001D0012100E00021084201D18C4302D0C3
:109CF0000120BDE8F0810020FBE7018811B942187E
:109D000092780AB101207047491C0829F7D3002036
:109D1000704710B50C460346FFF7EFFF00280AD046
:109D200018882188884205D10822A11C981CFCF7BC
:109D3000C8FB08B1002010BD012010BD03F022BDFA
:109D400070B50446FFF74EFF0546204603F017FAAC
:109D50004FF6FF7104468D4203D014B9284603F034
:109D600011FD204670BD000010B5FFF735FDFF283E
:109D700005D0044900EB400031F8200010BD4FF63B
:109D8000FF7010BD402600203EB5044603F04AFB9C
:109D90000EE0019920464631FFF7BBFF28B9019933
:109DA00020462A31FFF7B5FF10B1BDF808003EBDCF
:109DB0006A4602A9072003F009FB0028E9D14FF603
:109DC000FF703EBD10B50A4941600A4800F048FEE8
:109DD00058B902F013FB07491C238C22087404486D
:109DE0008C39001F006800F0A1FD002010BD0000AC
:109DF00014FE0200682C00202DE9F0412D4F0025B3
:109E000018B17D600120BDE8F0810879012258B1C8
:109E1000294E01280CD0274C4FF0020808340228A4
:109E200021D0032842D128E00A7103F06BF83BE00F
:109E30005FF0000000EB800116F82110022908D025
:109E4000401C80B20228F5D33A707D6041F61D5067
:109E5000D9E700EB800006F8205006EB8000406850
:109E600003F042F820E00D71A4F8048000230122E1
:109E70001248216801F0E4F916E00D71206803F042
:109E800033F80D4923682831498801EB810206EB3C
:109E90008201D1F804C0C4F800C04B60A3880B81D4
:109EA000A4F8048006F822500028ACD07D600E2073
:109EB000A9E7000030230020A42B0020E02300208D
:109EC0000146034802888A4200D000207047000003
:109ED000982500202DE9FC5F0E008346DDE90C4744
:109EE000C6F1000098469246814600D408460125F6
:109EF00003E000BF90FBFAF06D1C5045FADAA8456C
:109F000000D9454624B1002E01DB780700D5641E38
:109F1000B80702D5B8F1000F0AD0F80708D13CB154
:109F2000A54205D220215846641EFEF7F9FBF6E74C
:109F3000002E02DA4E462D2102E0780703D52B21B0
:109F40005846FEF7EDFB07F0030002280BD1B8F1ED
:109F5000000F08D13CB1A54205D230215846641EFD
:109F6000FEF7DEFBF6E7CDE90047434652463146B1
:109F7000584605F0F7FABDE8FC9F000070B50D46A5
:109F8000044600684FF4887102F0CEFA4FF49071E5
:109F9000206802F0C9FA4FF49271206802F0C4FA06
:109FA0004FF4A271206802F0BFFA20681249C0F88D
:109FB000041320686907000B40B2090E002806DA76
:109FC00000F00F0000F1E02080F8141D03E000F124
:109FD000E02080F8001420680121000B40B200F05E
:109FE0001F0291404009800000F1E020C0F880127B
:109FF000C0F8001170BD00001003020002460020EE
:10A000001268930702D0530702D47047500714D543
:10A0100002F00300012802D002280CD105E0C2F3AF
:10A0200083100B68801C184404E00223086803EBCB
:10A0300092521044086001207047086800EB925368
:10A04000C2F38910401CEEE70248007A002800D0D5
:10A0500001207047682C0020F0B58488A518944230
:10A0600000D82246A41AC288D6189A4200D81346AD
:10A07000D21A4B880788BB420CD34088834209D848
:10A080008888A04206D3A84204D8C888904201D349
:10A09000B04201D90020F0BD0120F0BD0021425C9A
:10A0A0000AB101207047491C1029F8D300207047DD
:10A0B000800701D000207047012070470A4810B582
:10A0C000807860B1002401E0022C06D02046FEF723
:10A0D000A3F8641C042CF7D310BD0324F6E7BDE8F5
:10A0E0001040FEF7B9B80000302200200348017983
:10A0F000C90702D00078FEF7EBB970473022002084
:10A100001721018041800021017141711B21817162
:10A11000C17170472DE9FE4F2B4D984691460F00B7
:10A12000824601D000260DE0684600F0D5FB6A4665
:10A130000021504602F08FFF2878009E10B99DF84C
:10A14000090098B14A463146504604F039FE0446AB
:10A15000014600225046FFF73FF90D2C32D008DCB3
:10A1600084B3082C2ED00B2C0BD12BE00520BDE89E
:10A17000FE8F112C10D0862C1AD0A4F54050023836
:10A1800020D00325B8F1000F04D0324621465046B6
:10A19000FEF7AAFE2846EAE73A4629795046FDF737
:10A1A00089FB4A46E9785046FDF784FB0025E9E73C
:10A1B0003A4629795046FDF77DFB4A46E9785046F4
:10A1C000FDF778FB2546DDE7902200202DE9F041E0
:10A1D000204F0E46154604463978FDF753FB0028FC
:10A1E00035D0204602F02EFF50B32046FFF7BCFDCD
:10A1F00080462046B978FDF745FB08B1012700E00D
:10A200000227204603F0C6F90028404602D0FFF797
:10A2100097FD0DE0A8F57F41FF3909D0072103F034
:10A2200037F8010004D0052902D0204604F02EFBA7
:10A230002B46324639462046BDE8F041FEF7F2BBD8
:10A240002A4631462046BDE8F041FEF761BDBDE833
:10A25000F08100008822002070B5094D0646E9789B
:10A26000FDF710FB044629793046FDF70BFB01464C
:10A2700022463046BDE870400123FFF74BBF000087
:10A28000902200202DE9F047394E002780463D46B8
:10A29000DFF8E090D6F804A057E003D00446D0F8E9
:10A2A0001C8035E099F8002002EB4201521CD2B22A
:10A2B00089F8002009EBC10199F80230091D9A4282
:10A2C00001D189F8005048680A780446012A12D062
:10A2D000022A02D0032A3BD108E004F015FF00B1A6
:10A2E0000127257434E00574C06900E07068002817
:10A2F000F9D170602CE0207C50BB88686060C86831
:10A30000A0600869E0604869A061F07800B165600C
:10A310006268B168184B501A20F07F40984202D210
:10A32000A168084406E0881AA16820F07F408142B5
:10A3300002D9081A206000E0256065600120A56050
:10A3400020742046E56104F0C1FEB8F10000A4D1FC
:10A3500099F8001099F801008142A3D117B97168EA
:10A36000514502D00120BDE8F0870020FBE7000046
:10A37000E8220020E4290020FFFF7F0030B585B0EF
:10A380000546002414216846FCF789F8A5F57F40AE
:10A39000ADF80250FF3815D02846FFF7B9FA98B14A
:10A3A0000B2815D0112811D0A0F54051023903D047
:10A3B0000146284604F056FA09482246C178284644
:10A3C000FDF778FA05B030BD0E2002E00124F3E776
:10A3D0000F208DF800006846FEF7C0FDECE7000096
:10A3E000502200200A4602498978FDF763BA00002E
:10A3F00050220020F8B5054600780C460026204281
:10A400000FD100208DF800006846FCF7A1FD2878E8
:10A41000204202D12043287001269DF80000FCF75D
:10A42000BBFD3046F8BD00002DE9FF410026234862
:10A4300000F013FB2148001F074600F00EFB204CE4
:10A4400060680090A56800E000986946284004EB29
:10A4500080000C30FFF7D2FD0028F5D101AA009949
:10A4600001EA050304EB8303491CDB6842F8203052
:10A47000401C00910228F2D3019800F0030001284B
:10A480000BD0022810D10198032101EB90500099C4
:10A49000BDF80A6001EB900005E00198BDF80A6084
:10A4A000C0F3831008440090384600F0D3FA08B196
:10A4B0000098606004B03046BDE8F081C0310020F3
:10A4C000A82D0020ACB04FF40041002001F02EFC7C
:10A4D00008B1FCF75BFC01F099FAFCF7BBFC08B192
:10A4E000FCF754FC01F040FD08B1FCF74FFC634958
:10A4F0000320FDF7A3FF08B1FCF748FC69460020E4
:10A50000FDF7CEFE08B1FCF741FC9DF800000228E3
:10A510007DD0002501F018FF08B1FCF737FC0024BE
:10A5200069460120009401F09DFD08B1FCF72EFC66
:10A53000684601F01BFE08B1FCF728FC03F030F977
:10A540009DF808004EA120F00F00401C20F0F00004
:10A5500010308DF80800112202A87CDF08B1FCF74A
:10A5600015FC00945020ADF80000A0200194ADF837
:10A570000200ADF804404FF4C870ADF8060068461C
:10A580007ADF08B1FCF702FC0021424800F0FBFA38
:10A5900008B1FCF7FBFBAC216846FBF780FF02200B
:10A5A0008DF8000001208DF802000621ADF81000A2
:10A5B0008DF87C008DF803104FF496703649229088
:10A5C000059144F2506023903448299031486946FF
:10A5D0002030FCF7DDFE08B1FCF7D8FB2D48012147
:10A5E0002030FCF7D2FE2E4801A9CDE900402948D1
:10A5F000143000F088FB08B1FCF7C8FBFDF7B4F994
:10A6000008B1FCF7C3FB27480090684600E032E041
:10A61000FDF780FA08B1FCF7B9FB1C216846FBF78F
:10A620003EFF4FF42030CDE900404FF470200290FF
:10A630001D48059003261D488DF80C600690ADF866
:10A640000E408DF810406846FDF7A4F808B1FCF7FD
:10A650009DFB174817A1008806EB004001F0F4FAB3
:10A660002846FCF7B1FA00BF01F0DEF90028FBD163
:10A6700001F0A2FCF8E701254CE7000095830200F9
:10A680004E6F726469635F427574746F6E6C65734C
:10A6900073000000342400202A22002049CC02004C
:10A6A0004DC00200397D02006DCC0200D789020046
:10A6B00024240020427574746F6E6C65737320449B
:10A6C0004655204170706C69636174696F6E2073C8
:10A6D0007461727465642E0070B5144682880E46EB
:10A6E00005462088111D0144921C994201D8FE2A7A
:10A6F00001D90C2070BD521C32542088FF21401C0F
:10A7000080B2208031542088401C80B22080811982
:10A71000288804F011FF2188084480B22080AA888C
:10A7200042B1A96841B13044FBF7A0FE2088A98856
:10A7300008442080002070BD072070BD2DE9F0473F
:10A74000C7880446181D16468946B0FBF7F1B0FBD2
:10A75000F7F207FB12009A193A44D21CB2FBF7F247
:10A76000DDF820A001E02468491E0029FBD13D1A34
:10A770008846B54216D818E0BAF1000F05D0211866
:10A7800009EB08002A46091D04E0204409EB0801F2
:10A790002A46001DFBF76AFE00202468761BA844A9
:10A7A000B74201D9354600E03D46002EE4D1BDE870
:10A7B000F087000030B5024659B101F0E3FA0021FC
:10A7C000074C09E004EB810315685B88AB4202D1BA
:10A7D0001160002030BD491C8142F3D3052030BDFB
:10A7E000F4230020F8B50F460178144605460129E8
:10A7F00001D1687830B12088821C9A422DD8012975
:10A8000002D006E00720F8BD69780144891C99420E
:10A8100023D8181A801E86B2ADF800602188B81CB3
:10A82000084469467DDF0028EDD12878022805D14B
:10A83000BDF80010B14201D809210AE00821012821
:10A8400005D16878B04202D8ADF8000001E0ADF85B
:10A850000060BDF80000FE2801D90C20F8BD228858
:10A86000401CB8542088401C80B220803954208875
:10A87000401C2080BDF80010084420800020F8BD56
:10A8800070B505460C004FF0FF0020D04FF6FF7664
:10A89000B5421CD00E48012241782846FDF70AF83F
:10A8A0002846FEF799FFFF2803D1FEF7B1FFFF28E6
:10A8B0000DD0084B00EB400203EB82014D8023F8E2
:10A8C000226022684A60A2880A81A2798A7270BDD9
:10A8D0006222002040260020034A00219268C0E93D
:10A8E00000218160704700009022002070B54FF673
:10A8F000FF750E46A84201D1002000E0401C84B242
:10A9000008E02146304603F014F908B1204670BD36
:10A91000641CA4B2FF2CF4D9284670BD10B5FBF717
:10A92000C4FC08B1002010BD112010BD10B531B11C
:10A93000B2FBF3F403FB14241CB1092010BD0E205C
:10A9400010BD01600021416081608281C3810846A1
:10A9500010BD70B50C460546FBF75CFC002802D024
:10A9600021882868084470BD10B50A8849888A4241
:10A9700003D1FBF791FC012010BD002010BD70B584
:10A980000C460546FBF76BFC002802D0618828685E
:10A99000084470BD10B50A8849888A4203D1FBF784
:10A9A00055FC012010BD002010BD01F01F03012245
:10A9B0009A40D243490900EB8100114600F059B892
:10A9C0000A4601F01F030121994010B552090C46B7
:10A9D00000EB820000F05DF8204000D0012010BDA7
:10A9E0002DE9F04180460D460024481E012101EB6F
:10A9F000501716E058F82400C04390FAA0F0B0FABF
:10AA000080F020280CD200EB4416AE4208D231462A
:10AA10004046FFF7D5FF0028ECD13046BDE8F08175
:10AA2000641CA742E6D82846F8E74A0950F82200F5
:10AA300001F01F0201219140084000D00120704721
:10AA400001F01F0301229A40490900EB81001146E1
:10AA500000F029B8002100F017B8012100F023B858
:10AA6000012100F016B808B56A46FBF76AFC0098A9
:10AA700008BD08B56A46FBF74AFC009808BD08B552
:10AA80006A46FBF75EFC08BD08B56A46FBF73FFC6B
:10AA900008BD08B56A46FBF72DFC08BD08B56A4637
:10AAA000FBF71CFC08BD08B56A46FBF723FC0098C1
:10AAB00008BD08B56A46FBF751FC009808BD38B5DB
:10AAC000044600258DF800506846FCF741FA2168DD
:10AAD0006268086890420ED9401E08600178A38A17
:10AAE000E26801FB0325227A2168101AC0B20A79B4
:10AAF000824200D208719DF80000FCF74DFA28460A
:10AB000038BD38B5054600208DF800000C46684673
:10AB1000FCF71EFAE868A98A201AB0FBF1F12A684E
:10AB20001068431C136001709DF80000FCF734FAB4
:10AB300038BD10B530B1017A42680368891AC9B2CC
:10AB40001A6006E00E2010BD03681A68541C1C60D1
:10AB50001170491EC9B2F7D2006800210171084680
:10AB600010BDC20800F007030120895C984008402E
:10AB7000704710B5C20800F00703885C01249C40B0
:10AB80002043885410BD10B560B10161172120F831
:10AB9000021B20F8021B1B2100F8021BFFF7B0FA72
:10ABA000002010BD0E2010BDF0B5858893B00C4676
:10ABB000002D39D1018800263E4F24293BD006DCE8
:10ABC000102909D011290CD0232958D14FE03A2956
:10ABD0000BD0552953D129E00146204602F054F804
:10ABE0004DE0A01DFFF78CFA49E02246408934F879
:10ABF000061F814200D808466080172800D217201F
:10AC00006080106970B1607960B1D7E90001CDE969
:10AC10000301ADF80E506088ADF81000136903A968
:10AC2000104698476671267113B0F0BD0146204664
:10AC300002F07AF823E0011D2C2206A8FBF716FC8F
:10AC4000BDF81800BDF81C2004EBC0014A7322694E
:10AC5000AAB1D7E90423CDE90423ADF81200487B5B
:10AC60008DF814002269204604A9904707E0017A74
:10AC7000207B884200D201462846FDF7F5FEA07AE7
:10AC80000028D1D0E1882846A5DF012570B1112820
:10AC9000CAD001F029FC0246074808A1008813B079
:10ACA00005EB0040BDE8F04000F0D2BFA672E572AF
:10ACB000BAE70000ACFC0200F423002073645F627A
:10ACC0006C655F67617474635F65786368616E6704
:10ACD000655F6D74755F7265717565737428292081
:10ACE00072657475726E65642025732E0000000015
:10ACF00020B10278DE2A03D0082070470E2070476A
:10AD000041800020704760B159B10278DE2A0AD034
:10AD100009684160DE2101704FF6FF71418000201B
:10AD200070470E207047082070477FB50546002900
:10AD30004DD0002D4BD008780C46DE2847D1A8888E
:10AD40006188884202D1204604F0B6FC2888012898
:10AD500025D002283BD011283AD0512837D135F8D8
:10AD6000040F6188884232D1A978A81C02292ED10B
:10AD7000017A042903D0062901D0052927D1002111
:10AD8000009102228DF8002001914FF4C0720291CF
:10AD90000391ADF80420007A05280FD010E0297A3D
:10ADA0002046012913D1A988428891420FD101215F
:10ADB000017204B0BDE8704004F07EBCADF8041030
:10ADC00028886946B0DF002801D0616888477FBDC8
:10ADD000A88861888842FAD14FF6FF7060807FBDF5
:10ADE00000F180400068002800D00120704708B5BD
:10ADF00000F18040002101600068009008BD000063
:10AE000070B54FF010246169104D0126491C288847
:10AE100014D06269032101EB00400DA100F018FF7E
:10AE2000606913DF040007D0288814A106EB0040F6
:10AE300000F00AFF204670BD002070BD06EB004008
:10AE40001BA100F001FF042070BD0000242400209D
:10AE500053657474696E6720766563746F722074CD
:10AE600061626C6520746F20626F6F746C6F6164D7
:10AE700065723A2030782530387800004661696C78
:10AE800065642072756E6E696E672073645F736FA0
:10AE900066746465766963655F766563746F725F17
:10AEA0007461626C655F626173655F7365740000F5
:10AEB0004E6F20626F6F746C6F6164657220776192
:10AEC0007320666F756E640070B50C4D03210C4ADB
:10AED000288801EB00400BA100F0BAFE084813DF00
:10AEE000040008D02888012101EB004010A100F0E7
:10AEF000ABFE204670BD002070BD00002424002061
:10AF00000060020053657474696E6720766563742F
:10AF10006F72207461626C6520746F206D61696E60
:10AF2000206170703A2030782530387800000000B9
:10AF30004661696C65642072756E6E696E67207318
:10AF4000645F736F66746465766963655F76656375
:10AF5000746F725F7461626C655F626173655F7369
:10AF60006574000070B50B4C207808B185250FE0A2
:10AF70000020A06060602061E060074801F0F0FA06
:10AF8000054601F03BFA08B901F0D4FA012020701F
:10AF9000284670BD042900204988020038B50025E4
:10AFA0008DF800506846FBF7D3FF074CE068401E61
:10AFB000E060E06810B901F0E3FAA5709DF80000C8
:10AFC000FBF7EAFF38BD000004290020F0B5054674
:10AFD0000478154889B0164640F82420124A0869BA
:10AFE000121DA2F1080742F82400487F385520229C
:10AFF0006846FBF73BFA04942878385C48B10EB1F8
:10B000000A4A00E000226946281D01F039FD09B016
:10B01000F0BD0EB1064A00E00022694605F10C00C1
:10B0200001F000FCF3E70000B022002015F402005C
:10B0300061F202000FB408B50399002904D004AAF4
:10B0400000926A4600F00FF801B05DF814FB10B5ED
:10B0500082680446002A05D0D4E904032168984791
:10B060000020A06010BD2DE9FC4791460C008046F1
:10B0700076D014F8011B39B125290ED04046FDF7D2
:10B080004FFB20780028F4D198F80C00002867D0F6
:10B090004046BDE8FC47FFF7DABF002001222178D7
:10B0A0002B291BD02D2902D0302908D102E040F0F5
:10B0B000010001E040F00200641C002AEFD10025ED
:10B0C0002A290ED02178A1F130020A2A11D205EBEB
:10B0D000850201EB4205641C303DF1E740F00400BD
:10B0E000EAE7D9F800100B1DC9F800300968641CA4
:10B0F0000D44217800232E290BD114F8011FA1F152
:10B1000030020A2A05D203EB830201EB4203303BF3
:10B11000F3E76C290DD068290BD0692921D00BDC0D
:10B12000252918D0582931D063290ED0642915D18A
:10B1300017E014F8011FECE7702969D0732932D0A9
:10B1400075291BD0782909D120E0D9F80000011D0C
:10B15000C9F8001001784046FDF7E2FA641C90E758
:10B160006CE0D9F800100A1DC9F800200968CDE983
:10B1700000500A224046FEF7ADFEEFE7D9F8001076
:10B180000A1DC9F8002009680A2206E0D9F8001053
:10B190000A1DC9F8002009681022CDE90050404678
:10B1A00004F0E0F9DAE7D9F8001000270A1DC9F821
:10B1B00000200E68C00705D112E04046761C7F1CB7
:10B1C000FDF7AEFA31780029F7D104E0202140469E
:10B1D0006D1EFDF7A5FABD42C0D9002DF6D1BDE721
:10B1E0004EB13046FBF766F9074604E020214046A1
:10B1F0006D1EFDF795FABD4206D9002DF6D103E08C
:10B200004046761CFDF78CFA31780029F8D1A5E785
:10B21000D9F80000011DC9F800100568302140462A
:10B22000FDF77EFA78214046FDF77AFA08200021E2
:10B23000CDE90001034610222946B0E7BDE8FC87AE
:10B240002DE9F84F2B4E04009A4630884FF0010349
:10B250001546894603EB004024D0216800292BD0F5
:10B26000002D32D0626849464FF010071268A2F1F3
:10B27000010C1CEA090F11D198466A432046FBF7DE
:10B280007BFC00282AD0206853462A46066901B074
:10B2900049462046B446BDE8F04F6047164B17A21A
:10B2A000009721E00E210091134B1EA21FA100F078
:10B2B000DEFC0E20BDE8F88F082100910E4B26A27F
:10B2C0001AA100F0D4FC0820F4E7092100910A4BF0
:10B2D00024A216A100F0CBFC0920EBE700973188EF
:10B2E000054B214A08EB014010A100F0C0FC1020E2
:10B2F000E0E7000014240020FBFD0200616464729A
:10B300005F69735F706167655F616C69676E6564D3
:10B3100028705F66732C20706167655F616464727A
:10B3200029000000705F6673000000002573206331
:10B330006865636B206661696C656420696E2025B1
:10B3400073282920776974682076616C75652030D0
:10B350007825782E00000000705F66732D3E705FC8
:10B36000617069006C656E006002030038B503000F
:10B370000F484FF001054FF00E04008805EB004028
:10B3800009D061B119600C6801B0A446BDE8304035
:10B39000114618466047074B07A2009402E0054B90
:10B3A00007A2009408A100F062FC0E2038BD000046
:10B3B00014240020B0FD0200705F667300000000DE
:10B3C000705F617069000000257320636865636BBE
:10B3D000206661696C656420696E202573282920C8
:10B3E000776974682076616C756520307825782ED1
:10B3F000000000002DE9F04128B1016819B1C969C8
:10B40000BDE8F04108470D4D0D480024461B1427A8
:10B410000DE000BF04EB840005EB8000016829B15A
:10B42000C969884710B10120BDE8F081641CB6FBF2
:10B43000F7F0A042EED80020F6E70000E02300205D
:10B44000F4230020044801214174007A08B100204F
:10B450007047012070470000682C0020012801D0AF
:10B46000032808D10449002201284A7400D0002092
:10B47000087402F007BE7047682C002070B50246C1
:10B48000022801D0032A45D1234C207A002841D03C
:10B49000012833D0022831D120480023022A006835
:10B4A00002D0032A2AD11BE0E360017911B10129FE
:10B4B00024D10DE0D0E90565711B4FF48056B142EF
:10B4C00000D33146294481614569A9420ED015E077
:10B4D0000169491C0161426991420FD1237213E055
:10B4E000E168491CE160082908D9E3602372022A57
:10B4F0000AD00D21FDF7CEFC02F06AFD607C28B178
:10B50000BDE8704000F080BF0021F3E7BDE8704067
:10B5100002F0B8BD70BD0000682C0020542300204C
:10B520002DE9F84F3A4D04008B4628884FF001066C
:10B53000DDF828A0984691464FF00E0106EB00403A
:10B540001AD0B9F1000F1BD02168002920D00921A1
:10B55000B8F1000F25D062685368B8FBF3F703FB1E
:10B560001782002A21D02B4B2BA2009135A100F08D
:10B570007EFB0920BDE8F88F264B3DA2009102E03A
:10B58000244B3DA200912FA100F071FB0E20F1E7AA
:10B59000082100911F4B3AA22AA100F068FB082065
:10B5A000E8E71C4B39A20091E0E75846FBF7DEFACA
:10B5B000102798B14846FBF7D9FAB0B14246594630
:10B5C0002046FBF7D9FAB8B1CDF800A02068434671
:10B5D0004A46C56859462046A847CBE700972888C1
:10B5E0000C4B06EB00402AA20CE000972888094B80
:10B5F00006EB00402CA205E000972888054B06EBDF
:10B60000004032A20FA100F032FB1020B2E7000090
:10B6100014240020E8FD020021286C656E202520FE
:10B62000705F66732D3E705F666C6173685F696EF4
:10B63000666F2D3E70726F6772616D5F756E6974B3
:10B6400029000000257320636865636B20666169CB
:10B650006C656420696E20257328292077697468D9
:10B660002076616C756520307825782E000000000A
:10B67000705F667300000000705F7372630000000B
:10B68000705F66732D3E705F617069006C656E005F
:10B69000616464725F69735F616C69676E6564336E
:10B6A0003228646573742900616464725F69735F32
:10B6B000616C69676E65643332282875696E74330E
:10B6C000325F7429705F7372632900006164647271
:10B6D0005F69735F77697468696E5F626F756E64C6
:10B6E0007328705F66732C20646573742C206C65FE
:10B6F0006E29000070B541EA4201DDE904564FF0C1
:10B70000A04441EA830141EA052104EB800041EABB
:10B710000641C0F8001770BD70B541EA4201DDE98D
:10B7200004564FF0A04441EA830141EA052104EBAD
:10B73000800041EA0641C0F8001770BD70B541EACB
:10B740004201DDE904564FF0A04441EA830141EA99
:10B75000052104EB800041EA0641C0F8001770BDE6
:10B7600070B541EA4201DDE904564FF0A04441EAD8
:10B77000830141EA052104EB800041EA0641C0F85B
:10B78000001770BD1CB5002100910B4601220191EC
:10B79000FFF7D4FF1CBD1CB5002100910B46012210
:10B7A0000191FFF7DDFF1CBD1CB500220B46009286
:10B7B00011460192FFF7C2FF1CBD1CB500220B46CB
:10B7C000009211460192FFF7CBFF1CBD1CB5002172
:10B7D00000910B46012201911146FFF7AFFF1CBDFE
:10B7E0001CB5002100910B46012201911146FFF783
:10B7F000B7FF1CBD4FF0A04202EB8000D0F800273D
:10B8000022F44032C0F80027D0F8002742EA014174
:10B81000C0F80017704701224FF0A043824011B1D9
:10B82000C3F808257047C3F80C25704718B5084BB6
:10B830006C4601441B68009306E000BF54F82030BA
:10B84000D3F81035401C08C28142F7D818BD00005B
:10B8500064FD0200034908B5084400210160006846
:10B86000009008BD0060004002494058012800D007
:10B87000002070470060004030B5124B01460020A8
:10B88000D3F81044224609E0157A854205D1401CC0
:10B890000A28F7DB4FF0FF3030BD5268002AF3D1A1
:10B8A000421CF9D00872D3F810242AB152684A60B9
:10B8B000D3F81024516030BD0022C3F810144A6040
:10B8C00030BD0000A82D0020F0B595B01C461546EF
:10B8D0000F4608461A9E00F025FB182109A8FAF722
:10B8E000DEFD0E96CDE909540023082203A938464F
:10B8F00000F02DFB05980690BDF81000ADF81C0077
:10B90000BDF81200ADF81E0000208DF8210003984C
:10B91000082600F00300012802D0022818D032E0E7
:10B9200003983346850AC0F3C2008DF820000398BF
:10B930000FA9C0F38314A200384600F008FB09A841
:10B94000009006AB22460FA9284600F047FA1AE0FD
:10B950000398840DC0F3C2008DF82000082C01D29A
:10B96000254600E0082533462A460FA9384600F050
:10B97000EEFA2E44641B09AB06AA29460FA800F074
:10B980007FF9002CEAD1384600F0D2FA15B0F0BDAC
:10B990007047012003F082BC084810B50178084ABE
:10B9A000515C19B1001D01F0F7F802E00C3001F014
:10B9B00005F8BDE81040002003F070BC68230020AB
:10B9C000AC22002008B5034A00924023024AFFF748
:10B9D0007BFF08BDB5E80200A82C00200A4A012917
:10B9E00002EBC00007D0022907D0032907D00429A1
:10B9F00007D000207047022070470420704700796C
:10BA000070474079704700005C09030010B5FFF7EC
:10BA1000C0FF04210348FFF72FFF024901204872AD
:10BA200010BD00007C2300202DE9F04F8DB0FCF705
:10BA300087FE18B100200DB0BDE8F08F7A4C4FF0B2
:10BA4000000BC4F818B4BFF34F8F60680290A5686C
:10BA5000D846284004EB800008E021680298814223
:10BA600001D86160E6E7284004EB80000C3002A9B1
:10BA7000FEF7C4FA0028F0D105AA029901EA0503ED
:10BA800004EB8303491CDB6842F82030401C029120
:10BA90000228F2D3059800F00300022802D0012802
:10BAA0004ED0A9E005985022810D8946B2EB905FF7
:10BAB00000D850210E4666F39F50059008315B4830
:10BAC00000F0E7F9070079D000F02CFA434608228D
:10BAD00005A9384600F041FA029908F1080A294000
:10BAE000681A8000001D864223D94F4D0C3530B1B5
:10BAF000C2B204EB8101301A90460C3104E02946B1
:10BB0000F2B2002590462846C6B25346384600F0A9
:10BB100024FA0AEB08032DB1324629464FEA070002
:10BB200000F01BFA029909F1030001EB900002906A
:10BB30003BE004EB81015346324638460C31EFE7D7
:10BB40000598C0F38310062800D30620059960F3FA
:10BB50008911C1F38310801C05918100334800F0E6
:10BB600098F9070048D000F0DDF94346082205A9FE
:10BB7000384600F0F2F908F1080800260FE00298B4
:10BB8000434600EA0501401C04EB810102900422B7
:10BB900038460C3100F0E1F908F10408761C0598EC
:10BBA000C0F38310B042EAD847B1D4F81054D4F8A7
:10BBB000180468B1384600F0BBF92FE01CE0687A41
:10BBC000012804D12A6828463946126890476D68D2
:10BBD000002DF4D1384600F0ABF98DF800B068467E
:10BBE000FBF7B6F9D4F8180408B9029860609DF81C
:10BBF0000000FBF7D1F911E0D4F8104404E021680B
:10BC00002046896888476468002CF8D108480221DA
:10BC1000008801EB004007A100F016F8FCF790FD4A
:10BC200080F0010007E70000A82D0020DC090300D8
:10BC3000242400204261636B656E647320666C751A
:10BC4000736865640000000000231A4603F0B8B969
:10BC500008B5012300926A4603F0B2F908BD1CB58D
:10BC6000CDE9002302236A4603F0AAF91CBD3EB5C4
:10BC7000069C8DE81C0003236A4603F0A1F93EBD33
:10BC80002DE9F0470E4680461C46924608293ED8CC
:10BC900094F80C90002020731946104602F02AF9FF
:10BCA0000025B54206D218F805201AA12046FFF754
:10BCB000C1F903E019A12046FFF7BCF96D1C082D5E
:10BCC000EFD317A12046FFF7B5F90025B54210D2F2
:10BCD00018F80570FAF7C6FB0068C05D10F03E0F5B
:10BCE00001D03A4600E02E220EA12046FFF7A2F92D
:10BCF00003E00DA12046FFF79DF96D1C082DE5D34B
:10BD000001222146504602F0D7F884F80C90BDE895
:10BD1000F08700002025303278000000202020002D
:10BD20007C0000002563000020000000104810B5D2
:10BD3000FF218160002101604160C0F81814C0F843
:10BD4000141480F820140B4800F0F0F800280DD1EE
:10BD500009480A490A4B401AC108002003E000BF05
:10BD600023F82000401C8842FAD3002010BD0000B8
:10BD7000A82D0020DC090300DC0903005C09030096
:10BD8000F423002002480349401AC008704700000D
:10BD9000DC0903005C09030013B56846FEF70AFDE1
:10BDA00008B100201CBD0248009950F831001CBDAC
:10BDB0005C09030070B508480125D0F8104480F8EC
:10BDC000205405E065722168204649688847646808
:10BDD000002CF7D170BD0000A82D00202DE9FF47F1
:10BDE00081460C9D00200C462F7B287398461646F2
:10BDF0002946184602F07EF8072E42D2DFE806F008
:10BE000004090F161F2A360049462846FFF712F983
:10BE100037E0494628462268FFF70CF931E0D4E9BB
:10BE2000002349462846FFF705F92AE0A06800905C
:10BE3000D4E9002349462846FFF7FCF821E0D4E97D
:10BE40000201CDE90001D4E9002349462846FFF765
:10BE5000F1F816E004F1080007C88DE80700D4E9FE
:10BE6000002349462846FFF7E5F80AE004F10800F8
:10BE70000FC88DE80F00D4E9002349462846FFF794
:10BE8000D9F800222946404602F016F82F73BDE883
:10BE9000FF872DE9F041858A80462D1F4819C01C77
:10BEA000B0FBF5F0C6B24046FEF709FE041E19D0FD
:10BEB0000020207101206071E58000272546761E54
:10BEC000C4F800800BE04046FEF7F9FD60B16179EF
:10BED000491C6171286005467F1CC0F80080B7428C
:10BEE000F1D32046BDE8F081204600F002F80020A2
:10BEF000F8E72DE9F041457901466B1E002201E08B
:10BF00000968521C9A42FBD30F680146002605E0DF
:10BF100038460C68FEF7F5FD2146761CAE42F7D395
:10BF2000BDE8F0810121001DFEF79DBDFEF701BEB9
:10BF300010B504460121001DFEF7BBFD10F0FF0FF8
:10BF400004D12046BDE81040FFF7D3BF10BD38B57F
:10BF500001240094FEF7F2FB38BD38B500240094AC
:10BF6000FEF7ECFB38BD00000F4910B5002048700B
:10BF7000091D0860BFF35F8F0C490D4800F070FA8F
:10BF80000A480C4A0121001FFAF752FF002809D184
:10BF900006480022001F4FF400410068BDE8104031
:10BFA000FAF782BF10BD00005C2300205CFE020097
:10BFB0009C2C002039C0020008B500208DF800003C
:10BFC0006846FAF7C5FFF1EE100A20F09F00E1EE97
:10BFD000100ABFF35F8F08494020C1F880029DF826
:10BFE0000000FAF7D9FF00F009FA08B141DF08BDF7
:10BFF00020BF40BF20BF08BD04E000E070B504468C
:10C000000C480121FEF74AFDBFF35F8F0025002891
:10C0100009D10120074E042C08D0311F4A781AB1EB
:10C02000BFF35F8F356070BD0C70487002F018FD73
:10C03000F6E700006023002003484078002802D083
:10C040000420FFF7DBBF70475C230020FAF79EBE99
:10C0500020B1034909680160002070470E20704735
:10C0600048000300FEB502460E460846FFF7F0FF03
:10C0700000286ED1002500950195012406208DF839
:10C080000020ADF8040002958DF80240694620209A
:10C09000326869DF2F4F48B100F026FA398802462E
:10C0A00004EB01432C491846FFF7D2FD00958DF8AB
:10C0B00001408DF80250019502958DF803506946B4
:10C0C0004020326869DF40B100F00EFA024638883D
:10C0D000224904EB0040FFF7BBFD00950195029556
:10C0E0008DF8004069460120326869DF48B100F0F0
:10C0F000FBF93988024604EB014319491846FFF75A
:10C10000A7FD4FF4B0600090019502956946A1200B
:10C11000326869DF48B100F0E7F93988024604EB7C
:10C12000014310491846FFF793FD009501950295CC
:10C130008DF800406946A020326869DF40B100F008
:10C14000D3F902463888084904EB0040FFF780FD28
:10C150000020FEBD2C240020F80703004008030047
:10C1600058070300A4070300040703002DE9F0416A
:10C170000446D0F8008060DF2168194D074641452C
:10C180001CD92888022606EB004016A1FFF75CFDAB
:10C190002888424606EB00401EA12368FFF75FFD9A
:10C1A000F006D0F80C012168800200F10050421A1C
:10C1B000288825A106EB0040FFF74AFD012467B15E
:10C1C000384600F091F9024628882AA104EB004085
:10C1D000FFF73EFD3846BDE8F0812E480470F9E7D0
:10C1E0002C240020496E73756666696369656E74F8
:10C1F0002052414D20616C6C6F63617465642066F0
:10C200006F722074686520536F6674446576696345
:10C21000652E00004368616E676520746865205272
:10C22000414D207374617274206C6F636174696F27
:10C230006E2066726F6D203078257820746F203004
:10C240007825782E000000004D6178696D756D20AD
:10C2500052414D2073697A6520666F72206170705B
:10C260006C69636174696F6E20697320307825781A
:10C270002E00000073645F626C655F656E61626CC6
:10C280006528292072657475726E65642025732E89
:10C2900000000000DB23002030B5144891B0007886
:10C2A000002820D05FF03405ADF8405010A903A855
:10C2B00061DF30B1052816D011B0BDE83040FAF783
:10C2C00065BD03AC0A49684600F0CAF807E000BF44
:10C2D000D0E9002120469047684600F0D8F802983F
:10C2E0000028E1D0F4E711B030BD0000DB230020CE
:10C2F0004C000300F8B5134C2078C0B10120A070A9
:10C3000002F054F9112814D0022002F067F9002538
:10C310008DF800506846FAF71BFE11DF06462570BF
:10C320009DF80000FAF738FE2EB13046F8BD08201F
:10C33000F8BD0020F8BDA57002F0FEFD032002F05C
:10C340004DF9F6E7D82300207CB5204C207808B1C1
:10C3500008207CBD0120A070002002F027F91128E0
:10C3600019D0002002F03AF919480026006801901F
:10C370008DF800606846FAF7EBFD164901A810DF5A
:10C3800005000AD0002020709DF80000FAF704FE96
:10C390002DB128467CBD00207CBD0120F3E7A670AE
:10C3A00066700721162002F0B7F808B1FAF7EEFC24
:10C3B0000721152002F0B0F808B1FAF7E7FC02F007
:10C3C000D7FD012002F00AF9E5E70000D82300209C
:10C3D000E0FF0200116D02000EB50749684600F04B
:10C3E0003FF805E0D0E900108847684600F04FF8B4
:10C3F00002980028F6D10EBDFCFF0200014800782B
:10C4000070470000D82300200548817819B10078D2
:10C4100018B1FFF76FBF08207047FFF795BF000006
:10C42000D82300201FB568464BDF30B1052814D053
:10C4300004B0BDE81040FAF7A9BC084901A800F013
:10C440000FF806E0D0E900210098904701A800F01D
:10C450001EF803980028E6D0F4E71FBD680003002B
:10C46000016009684160AFF3008010B5D0E9002198
:10C470005368994201D1002104E0D1E90034A3427C
:10C4800002D01946816010BD08314160F0E7816833
:10C4900000290BD0026892680A44826041684B68A8
:10C4A0009A4203D108314160FFF7DFBF70470000B7
:10C4B0000C4A10B502F594730EE0991AC91001EBFD
:10C4C000D171491002EBC1010C68844201D90B46BD
:10C4D00002E005D201F108029A42EED3002010BD1D
:10C4E000486810BD7CFE020000B5FFF7E1FF0028A0
:10C4F00000D1014800BD000068FE0200405800283D
:10C5000000D00120704708B50022425040580090EA
:10C5100008BDD0F80403084000D0012070474058FF
:10C52000002800D00120704708B500224250405832
:10C53000009008BD08480068012110F0010F08D1E3
:10C540004FF0E020E02280F80024C0F88012C0F80C
:10C55000001102480160704700E100E0180500404A
:10C560000649024600200B790BB1852070470A600E
:10C5700001220A7100224A7170470000B82200208F
:10C5800004490120086004480168C1F30041002902
:10C59000FAD170470C00004018040040002802D077
:10C5A000014980010847704781FD02002DE9F041F3
:10C5B0008846054601F034F9234E002828461AD053
:10C5C000FCF70AF9304490F848008009032802D0AB
:10C5D00001280ED007E04FF0A040D0F81005E84049
:10C5E00010F0010F05D003212846BDE8F041FFF708
:10C5F00001B90221F8E701F01FF9002822D02846EE
:10C60000FCF7EAF804464FF4807000EB84000F4F0B
:10C6100081B207EB8400D0F8102542F00102C0F887
:10C6200010250846FFF716F9B8F1000F0AD0284682
:10C63000FCF7D2F856F82000002803D00120A040D3
:10C64000C7F80403BDE8F08118290020006000400D
:10C650002DE9FC41DFF8BC80044608EB040000270C
:10C6600090F930001346C0170E46401C01D0082731
:10C670004CE0B0781946C0F340022046FCF788F839
:10C680000546401C41D0B078410719D4C0070AD0F4
:10C690004FF0A04000EB8401D1F8000720F0020029
:10C6A000C1F8000707E000217378204600910A4690
:10C6B0000191FFF731F8174920465431FEF759FA36
:10C6C000B078800718D51448317800EB8500D0F891
:10C6D0001025124B1A40C0F810254FF4F8524FF4B1
:10C6E000403302EA042203EA01410A43D0F810155C
:10C6F0000A43C0F8102509E008EB0500327810F86D
:10C70000481F41EA8211017000E004273846BDE865
:10C71000FC8100001829002000600040FFE0FCFFC1
:10C720004FF0A041D1F81015C14011F0010000D028
:10C730000120704770B5184D95F8580008B10820D1
:10C7400070BD0020411E2A18401CC0B282F8301073
:10C750002028F8D300242046FCF70CF8641CE4B22F
:10C760000C2CF8D300240D49E0206C6581F80004FE
:10C7700001264020891FC1F88002C1F800014FF452
:10C78000BE70FFF767F80649F007C1F8040385F8A3
:10C790005860204670BD00001829002006E000E027
:10C7A00000600040034890F85800002800D00120A5
:10C7B00070470000182900200121B1EB507F01D102
:10C7C000012070470020704738B50D4601F0DEFBB0
:10C7D000040014D000208DF800006846FAF7B8FB7A
:10C7E000207928B19DF80000FAF7D6FB112038BD5A
:10C7F0000120256020719DF80000FAF7CDFB002094
:10C8000038BD10B501F0C2FB002802D00021016044
:10C81000017110BD0149024802F068BD7429002071
:10C82000002000402DE9F0410546007916460F46EC
:10C8300000EB40012D4A01EBC00102EB810494F8AA
:10C840002A1011B10820BDE8F081294951F82010C3
:10C850002868FFF7B9FF08B11120F4E739462846E8
:10C86000FAF7B4FB66603869206030004FF00106CB
:10C870002FD03F7F4FF48E712868FFF744FE4FF4AE
:10C88000A2712868FFF73FFE28681A49C0F8041310
:10C8900028684FEA4711000B40B2002806DA00F082
:10C8A0000F0000F1E02080F8141D03E000F1E0200B
:10C8B00080F800142868000B40B200F01F0206FA4E
:10C8C00002F14009800000F1E020C0F88012C0F8B9
:10C8D000001128680421C0F800150020A061E06163
:10C8E00084F8290044F8140FA675ACE774290020D9
:10C8F00068FD0200800002002DE9F047054600793E
:10C900000B4600EB400101EBC000234901EB800422
:10C91000284600F043F810B11120BDE8F0874FF031
:10C920000008C4F82080A360626184F828804FF476
:10C930008E76474631462868FFF7E5FD28684FF0B8
:10C940000109C0F808902146286802F06BFC606875
:10C9500000BBD5F800A00EE094F8280008B10F271E
:10C9600016E031465046FFF7C9FD0028F4D02146B5
:10C97000504602F057FC216A60698142F1D331468A
:10C980002868FFF7BBFD0028F9D02868C0F80C9094
:10C99000C4F814803846C0E774290020007900EB01
:10C9A000400101EBC000044901EB80004069002810
:10C9B00000D0012070470000742900202DE9F047C5
:10C9C000044600794FF0000900EB400101EBC00084
:10C9D000254901EB80072068C0F80095786880B190
:10C9E00020682249C0F8081320680121000B40B2DA
:10C9F00000F01F0291404009800000F1E020C0F8E3
:10CA000080112068D0F80C25D0F81485D0F808657E
:10CA1000D0F810554FF0FF31C0F81415C0F80C15C0
:10CA20002068C0F80815C0F81015501C02D0104638
:10CA3000FEF7A8FEB8F1FF3F02D04046FEF7A2FE87
:10CA4000681C02D02846FEF79DFE701C02D03046BE
:10CA5000FEF798FE2068FFF7D4FE87F82A90C7F803
:10CA60000490BDE8F08700007429002084020200D1
:10CA70000149024802F0E6BCA02900200020004045
:10CA80002DE9F0410546164600790F46154A00EBA0
:10CA9000C00102EB810494F8201011B10820BDE818
:10CAA000F081114951F820102868FFF78DFE08B178
:10CAB0001120F4E739462846FAF7CCFA666038695F
:10CAC00020601EB1397F2846FDF758FA28680821F2
:10CAD000C0F800150020A061E0610121606184F8C8
:10CAE0002010DCE7A02900206CFD02002DE9F047B2
:10CAF00004460E460079204900EBC00001EB80059A
:10CB000017463046FFF758FE30B1204600F036F8A1
:10CB100020B11120BDE8F0871020FBE76F61AE6007
:10CB20004FF49076002731462068FFF7FDFC4FF464
:10CB3000AC7841462068FFF7F7FC2068AA6869696D
:10CB4000C0F84425C0F84815206801218160686854
:10CB500078B9B14649462068FFF7E1FC06464146F0
:10CB60002068FFF7DCFC0643F4D000B10F2700205B
:10CB700068613846CEE70000A02900200079054909
:10CB800000EBC00001EB80004069002800D00120CC
:10CB900070470000A02900202DE9F04704460079E5
:10CBA000274900EBC00001EB800720684FF0000927
:10CBB000C0F80095786880B120682249C0F8081351
:10CBC00020680121000B40B200F01F029140400993
:10CBD000800000F1E020C0F880112068D0F80C251A
:10CBE000D0F81485D0F80865D0F810554FF0FF3113
:10CBF000C0F80C15C0F814152068C0F80815C0F866
:10CC00001015501C02D01046FEF7C5FDB8F1FF3FCD
:10CC100002D04046FEF7BFFD681C02D02846FEF752
:10CC2000BAFD701C02D03046FEF7B5FD2068FFF754
:10CC3000E8FD87F82090C7F80490BDE8F087000071
:10CC4000A02900201003020010B550B103280CD118
:10CC50000220FBF7E7FB002807D0BDE81040FAF7F9
:10CC600095B8BDE8104001F039BF10BD007800282C
:10CC700007D104483B21008876DF002801D0FAF76D
:10CC800085B870472822002070B58D88027900EBA6
:10CC9000C5042273C97BA41D012902D0022904D135
:10CCA00001E0008800E0408820802188608881427F
:10CCB0000FD92846A5DF0126A0B1112814D0FFF70F
:10CCC00013FC02460A480BA1008806EB0040FEF761
:10CCD000BFFFA179E079814208D92846BDE87040BC
:10CCE000FBF7C2BE6671F4E72671F2E770BD000083
:10CCF000F423002073645F626C655F676174746322
:10CD00005F65786368616E67655F6D74755F726596
:10CD1000717565737428292072657475726E656407
:10CD20002025732E000000007CB506468D88C8883B
:10CD300006EBC504A41D172800D2172021888142C4
:10CD400000D8084660800020207121882846B5DF81
:10CD500050B1FFF7C9FB02460E480121008801EBE4
:10CD600000400DA1FEF774FF6079002810D13069F2
:10CD700000280DD01449D1E90201CDE90001ADF838
:10CD800002506088ADF80400326969463046904729
:10CD90007CBD0000F423002073645F626C655F67F4
:10CDA000617474735F65786368616E67655F6D74E5
:10CDB000755F7265706C7928292072657475726E62
:10CDC00065642025732E0000ACFC02007FB51A4D6F
:10CDD0008188AA8891422DD110F8061F022929D1F5
:10CDE0004188EA88914225D1017A042922D0062976
:10CDF00020D005291ED0841C002000900221019023
:10CE0000029003908DF80010297E19B101218DF850
:10CE1000061001E040F2FD10ADF80400A888694654
:10CE2000B0DF1128FAD0BDF80400002802D1204656
:10CE3000FAF7FCFE7FBD00009C28002048B1064A9E
:10CE40000168914205D140680449401802D0012888
:10CE500000D0032070470000DEC0ADDE02FEE10E10
:10CE60008A7D022A04D90289CB881A44D21C028105
:10CE70004289C988511AC91E418170472DE9F04184
:10CE80000D460221904600F58056298000F10804E5
:10CE9000144F1BE031462046FCF7E8FD40B1B8F1E5
:10CEA000000F02D0012288F80020022816D004E0EA
:10CEB000A0687969884200D9786128886188084427
:10CEC000C01C2880608804EB80040C343146204666
:10CED000FCF7DFFD0028DDD1BDE8F0814FF4806074
:10CEE0002880F9E71023002008B5002100910146B1
:10CEF0000823024A0248FEF713FB08BD98FD020012
:10CF0000E023002008B50020009004480823044ACC
:10CF100001680448FEF704FB08BD00003823002028
:10CF200090FD0200E02300202DE9F05F0025DFF8EE
:10CF30000891DFF808B12C464FF00308AA462F46A7
:10CF4000D9F80C0000EB07363046FFF777FF78B3CF
:10CF5000012847D0032862D100204FF4806200BF2F
:10CF600056F82010491C0ED004EB84010BEB810213
:10CF7000A8F10100566003221FFA80F80BF8212067
:10CF8000641CA4B24BE0401C9042E9D32C480168D9
:10CF900079B104EB840102200BF821000BEB810135
:10CFA0004E600881254828304480641CA4B205E006
:10CFB00007E00221066081804FF0010A45F001057B
:10CFC0002DE004EB840100220BF821200BEB810102
:10CFD00001F110024E6030460831FFF74FFF45F077
:10CFE0000205CDE7BAF1000F0CD0022004EB84015A
:10CFF000134A0BF821000BEB810112684A60641C94
:10D000000881A4B20E480022011D06603046FFF7D9
:10D0100035FF0B48808802280CD0082005437F1C70
:10D02000BFB2032F8CD3B8F1020F00D20025E8B2B3
:10D03000BDE8F09F0420F1E7E0230020A42B0020AE
:10D040003823002001494978FAF71CBC88220020C7
:10D05000002101F045BF30B585B00C4605218DF8A3
:10D0600000101546ADF80200FCF77EFEADF8040096
:10D070006846CDE90245FBF7A3FF05B030BD0000CF
:10D0800070B5054D06460024304655F824108847F3
:10D09000641C042CF8D370BDDCFC02003EB5104DBE
:10D0A000002400BF05EB041002F060FC641C022C9D
:10D0B000F8D30124502002210094CDE90110084941
:10D0C000084BB039A02201F1A00000F0EFFB08B13D
:10D0D00003203EBD0348401E847000203EBD00007A
:10D0E000F02700207522002000F06CB900F06CB928
:10D0F00070B504460025C168184A284602EB0013A3
:10D100009B688B4202D102EB001003E0401C022816
:10D11000F4DB00202178082904D0092908D013293C
:10D1200014D112E0617A89B980B102F02FFC0DE0D0
:10D13000617A59B950B100218160817B41F00201CF
:10D14000817307490120087003E001252046FFF79D
:10D1500097FF2846BDE8704001F020B8F027002076
:10D160007422002000F0E5B908B513889B000093F5
:10D170006B4600F05FF908BD002300F05BB938B5DD
:10D1800005460024204609E08178284600F080F812
:10D1900010B1052800D003240098401C0090694677
:10D1A000284602F0CFFB0028EED134B9284600F023
:10D1B000C4F910B1072802D00324204638BD072443
:10D1C000FBE71346002200F069B900002DE9F047A3
:10D1D0001F0015460E46814604D0072E05D0082EA6
:10D1E00016D102E00E20BDE8F0878DB1022D0FD8D8
:10D1F00000F0AEF960B14FF000083146484602F049
:10D2000087FB041E06D0207BA8420DD00F20EAE742
:10D210000720E8E7FF214FF6FF7002F079FB041EBC
:10D2200006D0A0F80090A670607BFF2802D00CE02A
:10D230001120D8E72946154800F00AFB0146204690
:10D240006173FF2913D04FF001082573617B0F48EC
:10D2500000F04CFB02000DD0ABB23146384600F076
:10D2600007FAB8F1000F0ED0082E05D00BE002F03F
:10D270007DFBDDE70320B6E738886FF0050101EBA1
:10D280008000796888800020ADE70000E02700205A
:10D2900070B5002402F03CFB05000BD0686820B19B
:10D2A00000F06FF9040000D00324284602F06EFB62
:10D2B000204670BD052070BD70B515460C46072987
:10D2C00003D0082C01D0072070BD02F021FB28B14B
:10D2D00005808470BDE8704002F0D8BA052070BDAA
:10D2E0007CB50D46072903D0082D01D007207CBD51
:10D2F000002602F00DFB040002D0606810B11CE0B3
:10D3000005207CBD617B0F4800F0F0FA02004FF071
:10D310000000009001908DF8025010D0237B294628
:10D32000684600F03DF9684602F09EFA211D684605
:10D3300000F010F90646092801D030467CBD0320D4
:10D340007CBD0000E02700204FF6FF7141800149BD
:10D3500009680847C4FC020030B587B01748FBF7DE
:10D36000B9FF10B1032007B030BDFBF7D5FE08B1FF
:10D370008620F8E700F0CEF9002002904CF2070476
:10D3800003900EE0694604A8FBF76EFF00988088C2
:10D39000A0F5404085B204A8FBF726FF284600F020
:10D3A00075F902AA04A92046FBF745FF0028E9D039
:10D3B0000349012008700020D5E70000CD8F02004E
:10D3C0006822002000F088B900F08CB970B586B0F2
:10D3D00014460E46054600F03BF940B105F54040C5
:10D3E00080B20F4A6946FBF726FF40B902E00120F0
:10D3F00006B070BD03A96846FBF736FF08B10020F0
:10D40000F6E7A57003984088208004986060039830
:10D410008088A0F5404030806846FBF7E5FEE6E7EF
:10D420006C220020024800214160816070470000AA
:10D4300068220020F0B587B01D46144607460E4608
:10D44000FF280AD8084600F003F930B103AA314694
:10D45000384600F0E5F840B902E0072007B0F0BD1B
:10D4600001A903A8FBF700FF08B10520F6E7A670A5
:10D4700001984088208045B18200286890420BD3F3
:10D4800002996068F8F7F2FF01E00298606003A873
:10D49000FBF7AAFE0020E1E70420DFE77FB586B0B6
:10D4A0001E460D460446FF282AD8A87800F0D0F87A
:10D4B00030B304F54040ADF80000A87803AA00F5A9
:10D4C0004040ADF802006868019028880290A97871
:10D4D000204600F0A5F80528089813D010B108A838
:10D4E000FBF726FF694603A8FBF7E2FEB0B1072869
:10D4F0001DD0082819D00E2817D003200AB070BDFF
:10D500000720FBE728B108AA694603A8FBF7DBFE62
:10D51000ECE7694603A8FBF7D2FEE7E71EB1314608
:10D5200003A8FBF798FE0020E8E71120E6E7862035
:10D53000E4E74FF6FF7000F0A9B810B5FF2801D955
:10D54000072010BD00F0A8F800F02EF8002010BD54
:10D5500000F0F4B870B504460D46807800F078F815
:10D5600058B121882846FBF7CBFE002804D00728B5
:10D5700005D0092800D0032070BD072070BD86208B
:10D5800070BD01B56846FBF7D3FE002800D003202C
:10D5900008BD00000149C978FAF774B98822002053
:10D5A0009BB200F065B8000070B51B4D8AB000203A
:10D5B000687000904FF6FF760190304603E02046F9
:10D5C00000F07CF8204600F087F80446B0421DD0F9
:10D5D00004F5404080B26A4602A9FBF734FE0A28EF
:10D5E000EDD004F5404080B2FBF756FD08280FD07F
:10D5F00000280BD005461422084905A8F8F736FF85
:10D60000ADF8184005A80795FFF79EFE0AB070BD5B
:10D6100001206870FAE7000068220020C8FC0200C0
:10D620007CB5054616460C46084600F011F8002069
:10D63000009005F54045019004F54044A8B2A1B220
:10D640006B463246FBF7F0FD002800D005207CBD7C
:10D6500007280BD0012809D0082807D0052805D0B5
:10D66000062803D0042801D000207047012070470D
:10D6700010B503EB83034FF6FF7404EA03138170C4
:10D68000DB1C99084260018010BD00000149FBF7D6
:10D69000ABB800001028002010B50446A0F57F406C
:10D6A000FF3807D004492046FBF79EF8A04201D17D
:10D6B000012010BD002010BD3028002010B5044608
:10D6C000044900F087FE03492046BDE810402031A0
:10D6D00000F080BE102800200149FDF707B90000C6
:10D6E0003028002070B50A49FDF700F904464FF6CE
:10D6F000FF7507E000F02CF838B105492046FDF72A
:10D70000F5F80446AC42F5D170BD204670BD00006E
:10D710001028002010B508484021F8F7C0FE4FF44B
:10D7200080742146044800F0D5F921460248BDE83E
:10D730001040203000F0CEB910280020FF2803D878
:10D740000146024800F0F5B900207047102800207B
:10D75000FF2803D80146024800F0EBB900207047CB
:10D760003028002070B500252C462146044800F0E2
:10D77000E0F9641CA4B20544FF2CF6D9284670BD1C
:10D780001028002010B50C46FCF726F8FF2804D01E
:10D79000024900EB400021F8204010BD4026002047
:10D7A0001CB500F071F908B1F9F7F0FA002000900B
:10D7B00001909DF8000020F07E0040F00100303024
:10D7C00020F080008DF8000007208DF80100102067
:10D7D0008DF802009DF8030040F003008DF803006F
:10D7E0009DF8040040F003008DF80400684600F046
:10D7F00053FB08B1F9F7CAFA034800F037FB0028D9
:10D8000001D0F9F7C3FA1CBD4DD902000068012808
:10D8100003D0022801D0002070470120704700008B
:10D820000449084490F93000082801DB01207047C2
:10D8300000207047182900200449084490F930005E
:10D84000082801D2012070470020704718290020C5
:10D850002DE9F0410F46060026D0306820B37068ED
:10D8600010B3FF2400251CE02946706800F039F948
:10D8700048B1FF2C00D12C46281B401CB8420ED1C9
:10D880002046BDE8F081FF2C06D108E02146304655
:10D8900000F040F8641CE4B2AC42F7D3FF246D1CE6
:10D8A000EDB2B068A842DFD8FF20EAE72DE9F041E9
:10D8B0000400DDE90705069E16D0A9B1A3B100FB5F
:10D8C00005F7974210D8C21DB6EBD20F0CD358B152
:10D8D00055B1E5602160C4E9013081B2184600F01D
:10D8E000F9F80020BDE8F0810720FBE770B50400DF
:10D8F0000D460DD0206858B1606848B1FF2D07D0A3
:10D9000000F017F920B1E168206805FB010070BD47
:10D91000002070BD70B504000D4611D020680028AD
:10D920000ED0606800280BD0FF2D09D000F001F95F
:10D93000002805D029466068BDE8704000F005B9B0
:10D9400070BD002901D001F0EFB87047F8B504466A
:10D9500000781E4D03260E281DD2DFE800F0071CBC
:10D960000F1C1D1C24351C331C352E35288818A18E
:10D9700006EB0040BDE8F840FEF766B96088F9F7AD
:10D9800063FF0246207A00902888638806EB0040F7
:10D990001AA1FEF76CF9F8BD002000906088694676
:10D9A000FFF7CFFFF8BDFBF799FB0828FAD0002856
:10D9B000F8D0BDE8F840F9F7E9B9BDE8F840002033
:10D9C000F9F702B92069F2E7A068F0E72424002003
:10D9D000436F6E6E656374656420746F20612070A0
:10D9E000726576696F75736C7920626F6E646564B9
:10D9F000206465766963652E00000000436F6E6EDB
:10DA0000656374696F6E20736563757265643A202F
:10DA1000726F6C653A2025642C20636F6E6E5F68B0
:10DA2000616E646C653A20307825782C2070726FB6
:10DA30006365647572653A2025642E0010B50F4C3D
:10DA40002168002919D04A7E002A16D00278082AB7
:10DA500002D0092A11D106E0007A01280DD1086907
:10DA6000401E086109D1F9F79DFF002805D0206804
:10DA70004169BDE810400220084710BDA8220020DF
:10DA8000FBF77ABAFBF778BA10B5FFF765FC88B9EF
:10DA9000FFF704FB70B901F049F858B901F064F9D7
:10DAA00040B9FBF735FE28B9FBF71AFF10B9FCF7B0
:10DAB000CBF808B1032010BD05484FF6FF718180F7
:10DAC00000218160417001210170002010BD000023
:10DAD00078220020002803D0C91DC908F8F7DFBC50
:10DAE0007047002809D001F0070301229A40D2B202
:10DAF00000EBD1001146FCF77DBC70472DE9F041E9
:10DB00000D46060013D0002401270EE004F00700A4
:10DB100007FA00F0C1B206EBD400FCF76BFC10B1C1
:10DB20002046BDE8F081641CA4B2AC42EED3284686
:10DB3000F7E740B100EBD10001F0070200780121C6
:10DB40009140084000D001207047F8B50400C1F3AF
:10DB5000C70501F007014FF0010000FA01F0C6B25D
:10DB60000FD0605D30420CD000208DF80000684678
:10DB7000F9F7EEF9605DB04360559DF80000F9F7E4
:10DB80000BFAF8BD2DE9F041044686B001278088E4
:10DB9000FCF728F86080207800263F4D082808D040
:10DBA000092820D04FF6FF780A2829D00B2853D116
:10DBB00058E0607A10B1012809D04DE0A86830B172
:10DBC000E168814203D1AE60A088A88016E0687841
:10DBD000E8B3A088A98888423ED1207A06283BD1A4
:10DBE00000F0C0FA38E0607A88BBA86878B3E168D2
:10DBF000814231D1AE60E868401EE860E6602BE00B
:10DC0000A878E8B14046FFF771FA4146404517D180
:10DC10000846FFF769FA404512D1AE7014216846F4
:10DC2000F8F73DFC0C208DF80000ADF80480ADF84D
:10DC3000028000272046FBF79FF96846FBF79CF916
:10DC4000687838B1A088A988884203D100E003E051
:10DC500000F088FA002F1CD006B02046BDE8F04145
:10DC6000FBF78AB9A8780028F6D0AE701421684670
:10DC7000F8F715FC0D208DF80000ADF80480ADF824
:10DC80000280A06802902046FBF776F96846FBF711
:10DC900073F906B0BDE8F0817822002008B5502263
:10DCA000ADF800200A466B46072100F001F808BDD8
:10DCB0007CB51D46164B1B7883B18AB185B12C8883
:10DCC0002346641EE61704EB967626F00306A41B93
:10DCD0001C1BE41C9C4205D007207CBD08207CBD99
:10DCE0000E207CBD0023009301932B880192DB1C46
:10DCF0009B08ADF800308DF802106A46FFF734FA41
:10DD0000BDF800104FF6FF7202EA810129807CBD48
:10DD1000782200200349097809B1FCF711B80820DE
:10DD2000704700007822002010B50C46064909789B
:10DD300029B134B1FCF718F82080002010BD08206C
:10DD400010BD0E2010BD0000782200202DE9FF4FED
:10DD50002A4883B09946007892468B46B8B14FF670
:10DD6000FF763046FFF7C2F9804600200090244835
:10DD700001AA062100680190CDF808D04046FFF7BF
:10DD8000F3F900256C1E3746072804D017E0082059
:10DD900007B0BDE8F08F0520FAE700200090A84208
:10DDA00001D305464746A04201D2044646464046B6
:10DDB000FFF79CF9804601AA0621FFF7D5F9D8B1F3
:10DDC0000528EAD0A8F57F41FF3901D00320DFE71D
:10DDD0000399002001B10F80BBF1000F01D0CBF8F7
:10DDE0000050BAF1000F01D0AAF80060B9F1000F9D
:10DDF000CED0C9F80040CBE70098D0E778220020C9
:10DE0000ECFC020070B5184E86B03078D0B101201D
:10DE1000B0704FF6FF742046FFF768F90546A04240
:10DE20001DD10020B07014216846F8F738FB0C2093
:10DE30008DF80000ADF80440ADF802406846FBF7ED
:10DE40009BF80EE0082006B070BD00BFFFF762FF30
:10DE500008B10320F7E72846FFF748F90546A54231
:10DE6000F4D10020EFE7000078220020084A117862
:10DE700021B1D178032903D30420704708207047CB
:10DE8000044B43F82100491CD1700020704700006A
:10DE900078220020502800200349097809B100F0B9
:10DEA00097BE08207047000078220020002801D08B
:10DEB000FBF762B87047000010B50C46017A0529DF
:10DEC00008D0407A38B1084808A102682046FDF71A
:10DED000B1F800E01AB106A12046FDF7ABF82046E4
:10DEE000BDE81040FDF7B3B8B4230020257300004F
:10DEF0000D0A000038B5C3880D46044633B114A09E
:10DF0000009015A216A12846FDF794F8217A05295C
:10DF10001CD0607A48B1A088FDF760FD164951F821
:10DF2000202016A12846FDF785F8A0880021FDF7DE
:10DF300033FF03461049207A143951F8202001B0EC
:10DF40002846BDE830400EA1FDF774B838BD00008A
:10DF50001B5B306D000000001B5B313B33316D00FB
:10DF600025734C6F67732064726F7070656420282E
:10DF700025642925730D0A00B423002025730000B1
:10DF80003C25733E2025733A200000000349884257
:10DF900001D1034870470020704700000020004076
:10DFA000C02200200146054810B50068FCF7D1FCEE
:10DFB00004461C21F8F773FA204610BD88FD0200C4
:10DFC000014602480068FCF7E5BC000088FD02003D
:10DFD000034802490068FCF7C7BC00005823002032
:10DFE00010FE0200F0B5254D254E85B004460027F1
:10DFF000686828B9214930680831FCF7C0FC6860BE
:10E0000001460078072817D2DFE800F01604080858
:10E010000E0E12002046FBF7EFFE02E0204601F054
:10E020003FFD040028D008E02046FAF7BBFDF8E7E2
:10E030002046FBF717FAF4E70F2414216846F8F797
:10E040002EFAA4F5E8501D3800D100240194694649
:10E050006868FAF7D5FE6846FAF70CFF07496F6063
:10E06000002408313068FCF77FFC044801210C30A3
:10E07000FCF71FFD0028BBD105B0F0BD1023002028
:10E0800088FD02002DE9F041234C0025234E207A23
:10E09000012730B92248311D0068FCF770FC306060
:10E0A00038B1022020723168087928B101281ED1C8
:10E0B00016E06560BDE8F081D1E90503C01A4FF4B0
:10E0C0008052904200D31046B7EB900F01D28208E5
:10E0D00000E001220869C9681844194429DF03E0F7
:10E0E000D1E90301084428DF58B1112812D00321D7
:10E0F0003068FAF7CFFE25726560BDE8F041FFF7A2
:10E1000067BF207C0028D5D1BDE8F0410021022066
:10E11000FDF7B4B92772CDE7682C00205423002006
:10E1200010FE020010B501210448FCF7A8FC0028ED
:10E1300003D1BDE81040FFF755BF10BD1C230020E0
:10E1400010B5074C201DFCF78BFC002806D1607C25
:10E15000002803D1BDE81040FFF794BF10BD0000B8
:10E16000682C0020084910B500231A46A1F10800C8
:10E17000FFF7ECFD30B1052804D0002002490C392E
:10E18000487010BD0120F9E78422002010B5104628
:10E190001A46F8F76BF9002010BD00002DE9F04792
:10E1A0001B4F82460026387886B0002821D00024F4
:10E1B000DFF86080A14600BF08EB0415A87B81074B
:10E1C00002D410EA0A0F1BD00126284601F05EFB9C
:10E1D000B0B14FF6FF71ADF802102988ADF8041008
:10E1E000862809D007218DF8001002906846FEF7B6
:10E1F00047FF06B0BDE8F08706208DF80000F5E780
:10E20000641C022CD8D3002EF3D187F80090F0E7DD
:10E2100074220020F02700202DE9F04707461E4811
:10E220001C46154600780E4670B185B17CB1DFF80A
:10E230006C804FF00009A08802282BD200EB8001EF
:10E2400018F8210010BB19E00220BDE8F087052076
:10E25000FBE720681FB181883A8891420ED11EB138
:10E2600001883288914209D18068286020686860FE
:10E270000A482830008928810020E6E7A088214646
:10E2800000F05EF80028E4D1C4F80090A088401C9B
:10E29000A080D0E70A20D8E730230020A42B00205C
:10E2A000F8B505464068244F0C46002648B323497C
:10E2B000CA68824225D80969814222D3FBF7F8FE59
:10E2C000F8B12889398988421BD1D5E900018A68CB
:10E2D000904216D10020A7F1280200BF00EB800376
:10E2E00002EB83035B688B4205D203F580538B42BC
:10E2F00001D9208011E0401C80B20228EED300201A
:10E30000F8BD268000960AE0009829688068884257
:10E3100005D100986860388928810120F8BD2088DF
:10E32000694600F00DF80028EED12088401C80B22C
:10E3300020800228E6D3E2E7CC2B0020E023002057
:10E3400070B50E4600EB8001134800EB8100446875
:10E35000306804F5805518B1418800EB810411E064
:10E36000083410E029462046FBF780FB20B1012845
:10E3700005D0022807D10DE00120346070BD60880F
:10E3800004EB80040C3429462046FBF782FB00286E
:10E39000E8D170BD002070BDA42B002038B50C461C
:10E3A0000021009101460423074A0848FDF7B8F808
:10E3B00008B10E2038BD064A04EB840102EB81014E
:10E3C00001200874002038BD8CFD0200E0230020ED
:10E3D000A42B00200A46FF2803D801461046FFF769
:10E3E000B4BB704710B596B050216846F8F757F89F
:10E3F000164C14A920688088FFF796FC002820D1CD
:10E40000BDF85000A0F57F41FF391CD06946FFF7E9
:10E4100045FC002815D117220D480DF10101F8F730
:10E4200025F80B481C2218300DA9F8F71FF8082012
:10E43000ADF85400206806490123808815AA3431BC
:10E44000B2DF16B010BD0F20FBE70000A8220020AD
:10E45000C82800200846704770B5012670044FF0A8
:10E46000E0210025C1F88001084C4010C4F84803A1
:10E47000C4F8080366602F20FEF790F8A660044CED
:10E480002F20A560FEF78AF8A57070BD001001402E
:10E49000E822002070B5054688690C4600284FF434
:10E4A000847128460AD0FEF72EF8D5F81805626A5E
:10E4B000E1688854606A401C606270BDFEF723F812
:10E4C000D5F8180570BD1FB501238DF80030CDE9D2
:10E4D0000121D0E90012684690471FBD1FB50123F6
:10E4E0008DF800308DF808100192D0E900126846CE
:10E4F00090471FBD10B50446064841792046F9F7FC
:10E50000C1F9002804D12046BDE8104000F01EBA31
:10E5100010BD00005022002070B50D460446F8F7EB
:10E52000F5FA70B12846F8F703FB68B16807000EEA
:10E53000002C0CDA04F00F0101F1E02181F8140D38
:10E5400009E042F2010070BD42F2020070BD04F128
:10E55000E02484F80004002070BD000038B50021DC
:10E56000012548B101280CD0032809D1FDF7E2FFAD
:10E57000BDE83840FCF712BD4FF0E020C0F88051F4
:10E5800038BD8DF800106846F8F7E2FC064C20789C
:10E5900008B9FCF7E7FCE068401CE060A5709DF856
:10E5A0000000F8F7F9FC38BD042900203EB5044608
:10E5B00009496846FDF754FF08E000BFD0E9002193
:10E5C0002046904730B16846FDF761FF0298002869
:10E5D000F4D13EBD11203EBDE4FF02003EB504462D
:10E5E00008496846FDF73CFF07E000BFD0E900217D
:10E5F000204690476846FDF74AFF02980028F5D16B
:10E600003EBD0000F0FF02002DE9FC4104460C3045
:10E6100000278046FBF7B8FB4FF6FF750646A84279
:10E62000208803D1FBF7A0FB064602E03146FBF74A
:10E6300085FB20880022012100F0C6F8AE4212D0EE
:10E640006A4607213046FEF797FD60B9019D95F8AF
:10E6500044003435C00705D1414605F11200FBF7EF
:10E6600058FB00B12F46002320881A46394686DF22
:10E6700005000BD0002320881A46314600F088F8A8
:10E680002088294600F002F9BDE8FC81002FFBD16B
:10E69000002320881A46314600F07AF820880022AC
:10E6A00041F20601FAF734FBEEE700002DE9FC41E8
:10E6B0001D46089C16460F46804644B16B46012213
:10E6C00007213846FEF782FD112801D010B1032042
:10E6D000BDE8FC8150210198F7F7E1FE0198067032
:10E6E0000198E5603430206001981830206101986D
:10E6F000401C60610748E061019940461131FBF719
:10E70000F5F90028E3D107213846FEF7E9FD052891
:10E71000DDD0DDE75C280020002835D002789107A5
:10E7200001D411062FD4C2F3021104292BD8930768
:10E7300003D5032901D1110625D5437881788B4271
:10E7400021D8072B1FD310291DD8C1784B071AD405
:10E750000079430717D40B0715D4030713D4D20746
:10E760004FEAC17201D042B10FE062B989070AD401
:10E77000C10708D1800706D407E0890705D4C1077F
:10E7800003D1800701D400207047012070470000AA
:10E7900070B50C4605466AB1002B12D0094801221B
:10E7A000C1782846F9F786F821462846BDE870402A
:10E7B000FBF7C4BA002B04D0BDE870400846FBF755
:10E7C000BFBA70BD88220020F0B5174D14460F4621
:10E7D0000A4685B006462978F9F76CF8002F1FD055
:10E7E0000CB1012200E0002269783046F9F762F8A6
:10E7F000012C17D00022A9783046F9F75BF80022E7
:10E80000E9783046F9F756F8142208496846F7F7D0
:10E810002DFEADF802608DF808406846FAF7C2FB9D
:10E8200005B0F0BD0122E6E78822002000FD0200CD
:10E8300010B586B0044614216846F7F730FE042070
:10E840008DF80000ADF802406846FAF7ABFB06B061
:10E8500010BD000002498969002900D008477047AF
:10E86000AC25002030B585B00C460546142206497B
:10E870006846F7F7FBFDADF8025068460294FAF7D8
:10E880006DFB05B030BD00003CFC020030B585B02A
:10E890000C460546142206496846F7F7E7FDADF831
:10E8A000025068460294FAF77DFB05B030BD0000C7
:10E8B00014FD020070B50D4C0020D2B22070201D56
:10E8C0000B4D0378EB5C1BB1001DFEF70FF902E066
:10E8D0000C30FEF711F808B1F8F758FA6078002804
:10E8E00002D021780029FAD070BD000064230020F6
:10E8F000AC2200200348002201490079F8F78EBFBE
:10E90000F5E40200502200207CB50E490E4C002296
:10E91000D1E90001CDE900016946A088FEF751FC6C
:10E920004FF6FF7507E00846FEF7E0FBA0800022E7
:10E930006946FEF746FCA188A94201D01128F2D110
:10E940007CBD000090FC02005C22002070B586B007
:10E95000064601250024FBF76DF8112812D005DCCE
:10E96000F0B1062828D0082808D125E0A0F54051AC
:10E97000023907D0A1F54071FF3924D00146304655
:10E98000FFF770FF2A46124D30462979F8F792FFBB
:10E99000697906B022463046BDE87040F8F78ABF74
:10E9A00014220C496846F7F761FDADF802600124B6
:10E9B0006846FAF7D3FAE5E700253046FBF7D4F9C5
:10E9C000FAF780FFDEE73046FBF7D8FCDAE7000015
:10E9D0005022002064FC02002DE9F0410746806AC5
:10E9E00014468846C8B3002531E000BFB96A05EB7C
:10E9F000450001EB8006B088801CFE2802D90C205F
:10EA0000BDE8F0812288401C08F802002088162208
:10EA1000401C80B2208008F800202088401C80B272
:10EA2000208000EB0801308800F086FD2188084432
:10EA300080B22080B28842B1B16871B14044F7F72A
:10EA400015FD2088B188084420806D1CEDB297F830
:10EA50002C00A842CAD80020D2E7FFE70720CFE762
:10EA600070B5194D194C07E00168207888470028D7
:10EA700029D01548FDF70BFDA8680028F4D1FDF753
:10EA800099F900BFFCF7D0FF0028FBD120780328BC
:10EA90000CD002280AD0FDF7B1FC00B133DF0C49DD
:10EAA00001200860BFF34F8F20BFFDE7BFF34F8FFA
:10EAB00008480168084A01F4E06111430160BFF3AE
:10EAC0004F8F00BFFDE770BD9C2C00205C23002011
:10EAD000000500400CED00E00400FA0510B5002030
:10EAE000F9F7A0FC08B1F8F751F9F9F7F5FB08B10F
:10EAF000F8F74CF9FDF7FEFB002803D0BDE8104005
:10EB0000F8F744B910BD000010B500F0ABF80548A7
:10EB1000002203494078BDE81040F8F77FBE0000AE
:10EB200059A202009022002000F016B910B5114839
:10EB3000FAF735FC0F48401CFAF731FC0D48801CF1
:10EB4000FAF72DFC0B48C01CFAF729FC0948001DF8
:10EB5000FAF725FC0748401DFAF721FC0548401E3E
:10EB60008179182903D00121C171002010BD032033
:10EB700010BD00009122002010B50078114C0A2829
:10EB800013D004DC082810D009281AD10DE00B2876
:10EB90000BD0132815D100220B49A079F8F73EFEBF
:10EBA00000220A49A078F8F739FE00220649607968
:10EBB000F8F734FE6078BDE8104000220349F8F70A
:10EBC0002DBE10BD9022002051D0020059A202009B
:10EBD00070B50B4C05004FF001060CD0FFF79CFD03
:10EBE00058B1286820612879207504F11000A060D0
:10EBF0002670002070BD0020F9E7072070BD0000DE
:10EC00009022002010B504460078052802D0122872
:10EC100021D105E06088A168BDE8104000F060B92E
:10EC20000F480021806880B10D48237A10300078A9
:10EC300000F0010203B101239A4206D3627AC0F3C5
:10EC4000400002B10122904200D2012160880123DC
:10EC50000022FBF75FFA2046BDE81040FAF7B0B992
:10EC60009022002030B50446008885B014284FD08B
:10EC70000ADC11282CD0132828D134F8040FF8F717
:10EC8000E3FD01282FD038E0192847D01A281DD1DC
:10EC9000A088FEF7D7F9002818D1A088F8F7AEFDB4
:10ECA0000028A0884BD02A4900220978F8F702FEF4
:10ECB00002208DF80000A088ADF8020000208DF839
:10ECC00008008DF809006846FAF76CF905B030BD08
:10ECD000207A3D2804D04FF48851A088002224E0F7
:10ECE00041F23D01F9E72079C00701D0012200E09F
:10ECF000022220880121FFF767FD34F8045B14220B
:10ED000014496846F7F7B2FBADF802500294DAE70F
:10ED100005B0201DBDE83040FFF776BC217A201DEC
:10ED200041B14279008802F0030205B0BDE83040ED
:10ED3000FBF74CBA05B0BDE83040F8F7D1B905B0E3
:10ED40000122BDE8304041F20601F9F7E1BF0000C1
:10ED5000882200203CFD02000A7802490979F8F770
:10ED6000A9BD00008822002010B51448FAF70EFB58
:10ED70001248401CFAF70AFB1048801CFAF706FB01
:10ED80000E48C01CFAF702FB0C48001DFAF7FEFA09
:10ED90000A48017818290FD0417818290CD08178B9
:10EDA000182909D0C178182906D00179182903D06B
:10EDB00001214171002010BD032010BD88220020D8
:10EDC00070B50C460546F8F73FFD012802D043F226
:10EDD000020070BD21004FF00000FAD028467EDF0F
:10EDE00070BD00002DE9F74F8AB0924688460A9818
:10EDF000F8F72AFD06464FF6FF7900244D462746D0
:10EE00000A98FEF7C7FB8346202101A8F7F747FBC6
:10EE1000012E01D0DEB105E02F48002201790A98C9
:10EE2000F8F748FDB8F1000F16D098F80000C007B9
:10EE300014D00A98FAF798FF0546484516D1FEF710
:10EE400091F9054648450ED04FF0010B0CE043F216
:10EE500002000DB0BDE8F08F852721E01F48CDF8F6
:10EE600010A008901CE003246CB121E0012E0AD10F
:10EE70000A98F7F7F9FE30B90A98FFF7D9FC0A9813
:10EE8000F7F7F2FE50B101A80090534632462946EA
:10EE90000A98FFF70BFC040002D009E0852712E076
:10EEA000012E10D001AB002239460A987FDF0446BC
:10EEB00054EA07000DD000225B4629460A98FFF766
:10EEC00067FC2046C5E701AB424639460A987FDF1A
:10EED000EDE70122F0E70000882200205C280020F6
:10EEE0003EB505460C466846FBF7F6FC6A462146E9
:10EEF0002846FEF7B0F809480099C2682846FFF78F
:10EF000071FF0446014601222846FAF765FA2146B8
:10EF10002846009AF9F7E8FF3EBD00009022002045
:10EF2000002805D10349012048700020F9F778BC7A
:10EF3000704700000429002010B51620F7F7E6FD01
:10EF400048B10A4882684FF4800152B1016821F447
:10EF50008001016010BDBDE8104042F20100F7F7EA
:10EF600015BF4FF0E020C0F8801110BDF02A00203E
:10EF700010B51620F7F7CAFD80B10F4890F80004CD
:10EF80004009F7F7D5FD60B10C4882684FF4800165
:10EF90006AB1016841F48001016010BD42F20100D4
:10EFA00001E042F20200BDE81040F7F7EFBE4FF07B
:10EFB000E020C0F8001110BD16E000E0F02A0020AB
:10EFC0002DE9F84F204D9246894606469846012283
:10EFD00069461846AF68F9F75BFB58B30098002103
:10EFE0000446801C09E000BF00EA07035AF821200C
:10EFF00005EB8303401C491CDA604145F4D34FEA1A
:10F00000164AF9F75BFE4AEA0041601C384005EBFE
:10F0100080003C4005EB8402C160D06866F3C50007
:10F0200068F3891069F39F2020F00300401C20F052
:10F030000400D06095F8200402E000BFFCF7F4FC67
:10F040000028FBD1BDE8F88FA82D00202DE9F84F4E
:10F050001D4C00256846D4E901A6F9F739FE0027C2
:10F0600038B30023009A61681CE0D1F800C008465C
:10F07000944503D9ACEB02020A6015E0A2EB0C0246
:10F0800063440760D0F80CC0C1698146BCF1000F31
:10F0900008D006EB030828F07F48C0E9018CC9F8C6
:10F0A0001C5005460029E0D128466160FBF7EAF8CC
:10F0B00003E02846FBF7E6F810B15046F9F7D2FB1B
:10F0C000E770BDE8F88F0000E82200200D4B10B576
:10F0D000596831B102680C68A24204D8A21A0A60C9
:10F0E000C161586010BD0B4603E00B46C969121B95
:10F0F00021B10C689442F8D3A41A0C600260C1617B
:10F10000D86110BDE82200202DE9F041144E776847
:10F110003D462C4603E0844204D02546E469002C99
:10F12000F9D11BE0D4B1A5420BD1F869706040B9A8
:10F130000C49012088600021B160F0702F20FDF79C
:10F140002DFA2168E069E86110B10268114401609C
:10F150007068874202D00120BDE8F0810020FBE703
:10F16000E8220020001001407CB5064600240D4630
:10F170008DF800406846F7F7EBFE01A800F0AEFA04
:10F1800070B10570094946609DF8040048709DF80B
:10F190000000F7F701FF1420F7F7B6FA20467CBD10
:10F1A00004249DF80000F7F7F7FEF7E7E4290020B4
:10F1B0002DE9F041194D6C68002C2CD0184800271F
:10F1C0000068A968B846401A20F07F462068B0421F
:10F1D0000CD82146361A0744E469087C20B181F82E
:10F1E0001080886949698847002CEFD129786878B0
:10F1F000814206D1401CC0B26870022801D185F856
:10F200000180064869780C3040F82170BDE8F04173
:10F210001420F7F779BABDE8F0810000E822002059
:10F220000415014070B50C4605464FF48E71FDF78C
:10F230006AF9216AA068415C206A401C2062C5F816
:10F240001C1570BD1FB500228DF800200291816849
:10F2500001914261D0E90012684690471FBD00004D
:10F260001FB50A4601788DF8001041680191017AB6
:10F270008DF80810C0680390044850F82210001F51
:10F2800050F82220684690471FBD0000B42200209D
:10F2900001490120087070476423002010B588B030
:10F2A000044620220E496846F7F7E0F80620009051
:10F2B000C01F0190029003904FF0EB7006900CB1CC
:10F2C000084A00E0002269460748FBF77FFE08B1C4
:10F2D000F7F75CFD0448001F447008B010BD000043
:10F2E000B0FF020091F20200682300202DE9FF47E1
:10F2F0000C4605464FF40071FDF70BF901274FF45A
:10F300000178002618B34FF4927949462846FDF754
:10F31000F5F8E0B149462846FDF7F5F8C5F8088349
:10F3200094F8290000B96F6002208DF80000D5F82C
:10F330008004C5F880040390A0690290E068019001
:10F34000A661E661D4E900126846904728E00421EE
:10F350002846FDF7DEF818B34FF484712846FDF710
:10F36000CDF8E8B121462846FFF794F8616AA06914
:10F37000884215D1E06938B1E268616AA06120690C
:10F38000E6616662E06008E094F8290000B96F6009
:10F39000C5F80883A661E268616A2046FFF793F822
:10F3A0004FF48E7841462846FDF7A8F878B1206AD8
:10F3B0006169884202D294F8280020B34146284669
:10F3C000FDF7A1F8616911B12046FFF73BFF4FF44B
:10F3D000A27841462846FDF791F8002818D041460A
:10F3E0002846FDF790F894F8290000B12F60A06935
:10F3F00000280DD0A661E268616A04B02046BDE82D
:10F40000F047FFF760B821462846FFF70BFFDEE71D
:10F41000BDE8FF871FB50A4601788DF800104168E6
:10F420000191017A8DF80810C0680390044850F8E3
:10F430002210001F50F82220684690471FBD000090
:10F44000B42200202DE9FF410C464FF49277054687
:10F450003946FDF764F80026C0B139462846FDF765
:10F4600063F802208DF80000D5F88004C5F8800408
:10F470000390D5F83C058DF80800E0680190A6617E
:10F48000E661D4E900126846904723E04FF488779C
:10F4900039462846FDF743F8E0B139462846FDF7DE
:10F4A00043F8D5F83C15A069884213D1E06960B1F2
:10F4B000E268D5F8000220F02000C5F80002E069FB
:10F4C000A0612069E661E06001E0A661E268204693
:10F4D000FFF704F84FF4A27739462846FDF71FF8E6
:10F4E00060B139462846FDF71FF8A06930B1A66122
:10F4F000D5F83C152046E268FEF7F0FF4FF4907710
:10F5000039462846FDF70BF8002813D0394628461F
:10F51000FDF70AF8606900280CD0D5F84C058DF885
:10F5200000608DF80800A06801906661D4E90012BF
:10F5300068469047BDE8FF810870000A48700220C5
:10F540007047000010B514210448F6F7A8FF0448DE
:10F550000068FBF7E3F9002010BD0000682C0020D4
:10F5600010FE02002DE9F05F8346DDE90A4A994664
:10F5700090460D460846012703E000BFB0FBF8F0B7
:10F580007F1C4045FAD2B94500D94F465FEACA70A0
:10F5900012D18CB15FEA8A7002D5B9F1000F01D0A7
:10F5A000202607E0302605E031465846641EF9F76C
:10F5B000B7F80CB1A742F7D35FF00106B9F1010F1C
:10F5C00002D9A9F1010903E0B5FBF6F0404502D3E9
:10F5D00006FB08F6F2E7DFF83C9000BFB5FBF6F05B
:10F5E00000FB165519F800105846F9F799F8B6FBC4
:10F5F000F8F6002EF2D15FEACA7009D0002C07D0CD
:10F60000A74205D220215846641EF9F789F8F5E78C
:10F61000BDE8F09FA0FD0200034800220149807868
:10F62000F8F7FCB8258B020050220020F8B50546FB
:10F6300080B2FAF745FC040013D0154E207A00275B
:10F64000317B88420ED2A8B204F10A0175DF28B1DD
:10F65000112806D0BDE8F840FFF7FCB8207A401C1E
:10F660002072F8BD2772307C38B1A8B23B2176DF1A
:10F6700018B1082801D0FFF7EDF871690029F0D022
:10F680008DF80070ADF8025068468847F8BD00005C
:10F69000AC250020417939B190F8B21021B990F829
:10F6A000B40008B1012070470020704701460148AE
:10F6B000FBF7BBB9C825002030B40446007A002807
:10F6C0000AD06088002166DF28B1112802D0616865
:10F6D00030BC08470120207230BC70470A494A7884
:10F6E0008B78521CD2B2934200D100220B78934205
:10F6F00001D1002070470270487800EB400001EB18
:10F70000C000001D70470000E42900202DE9FC41E5
:10F710001646DDE90854CDE900541F468046022212
:10F7200000F00CF8002807D1CDE900543B46102228
:10F730003146404600F002F8BDE8FC812DE9FC5F4F
:10F740000026DDE90C4B994692468E468046278876
:10F75000354630E0D8F80400002200EB8500694609
:10F760000068019001A864DF002830D19DF80000F6
:10F7700050451FD10EB1002100E00221228808442B
:10F780001118594522D846B9521C90B2208009F868
:10F7900000E02088401C20800126218801A801EB80
:10F7A0000902694664DF002811D120889DF8001005
:10F7B000084420806D1CB8F80000A842CADC56B18D
:10F7C0002088C01B401E80B2FF2802D90C20BDE853
:10F7D000FC9F09F807000020F9E710B5042817D2AC
:10F7E00009B1032400E00024F8F7C4FC4FF0A04165
:10F7F00001EB8000D0F8001721F44031C0F8001769
:10F80000D0F8001741EA0441C0F80017002010BDED
:10F81000062010BD002070472DE9F84F114D884695
:10F8200081461E4617466946DDF828A02868FBF782
:10F8300090F8040013D01C21F6F731FE002020714F
:10F84000C4F80090C4E90486C4E902A769462868A0
:10F85000FBF7A0F8FEF774FC0020BDE8F88F042049
:10F86000FBE7000010FE020082780121012A0BD084
:10F87000062A09D0072A06D0082A06D141688988B5
:10F880000931890800E01421018070471CB5044645
:10F89000002000900190A0788DF80200617B1A484A
:10F8A000FEF724F8020017D0237BA1786846FDF705
:10F8B00077FE6846FFF7D8FF208804F10803694601
:10F8C0006268FDF7EBFD48B1072806D001210F4A19
:10F8D000112808D086280FD003201CBDA17B21F061
:10F8E0000301A1731CBDA07B20F0010040F00200C9
:10F8F000A073117000201CBDA37B23F0020343F012
:10F900000103A37311701CBDE027002074220020A6
:10F9100038B505460C46002001E00098401C0090D8
:10F920006946284600F00EF800280AD08178A142E6
:10F93000F3D1817B8A07F0D4C907EED18168002911
:10F94000EBD138BD10B5084B0A6809E003EB02148F
:10F950002488844203D103EB02100A6010BD521CBC
:10F96000022AF3D3002010BDF02700204FF6FF71CC
:10F970000180FF2181704173817B21F0030181733C
:10F9800000210173416081607047000070B5054639
:10F99000002406E0687B2044C1B20648FDF7BAFFA8
:10F9A000641C287BA042F5D82846BDE87040FFF7CC
:10F9B000DDBF0000E02700202DE9FC470646364861
:10F9C0009846144600780D464FF0000978B37DB391
:10F9D0002888A0F57F41FF3931D0688848B368682E
:10F9E000FAF766FB68B374B32088ADF80000678847
:10F9F00001A8FEF7D7FA04002FD084F800804FF05A
:10FA0000000A84F816A0BDF80000A0826868206192
:10FA1000214801210C38FBF726F8E0602888208176
:10FA20006888A080E780B8F1030F1DD020E001E0D6
:10FA300003E004E00220BDE8FC870520FBE704208A
:10FA4000F9E70320F7E7FFE72889694687B23846D8
:10FA500000F0ACF80028EED1CAE7BDF80010384637
:10FA600000F098F80820E6E70420A0753068A0614F
:10FA7000A4F80A9001A8FEF7A3FA46B1C6F804A0BC
:10FA8000E1680648316086F80AA000893081FEF7F7
:10FA900049FB0020CFE7000030230020CC2B0020C2
:10FAA0002DE9F8430D46898A374A01EB810102EBC3
:10FAB000810630B129463046FDF7D2F90120BDE874
:10FAC000F88331897068002400EB81072E48A97DF6
:10FAD000A8384FF00E0807294ED2DFE801F00D2DAF
:10FAE000162404404A004460A96901602648274959
:10FAF000A838FEF7D5FB30B10220A875042339469B
:10FB00002A1D009423E00A20D9E728692A4608B173
:10FB1000032000E001209075042305F10C0207F199
:10FB20000801009413E00120A8750094E88807F10B
:10FB30000C0183002A690AE028782A4603280CD0A1
:10FB400006209075042305F10802391D0094104821
:10FB5000FBF7E6FCA8B144460FE00520F1E70621DB
:10FB6000A9750A4940680988FEF718FC040004D109
:10FB700007E041F61D5400E00F2429463046FDF70A
:10FB80006FF920469BE70000A42B002010230020E3
:10FB9000E023002001EB8102034901EB82014A8945
:10FBA000101AC01E48817047A42B002070B5C01CDD
:10FBB00082B240F2FE30824201D3092070BD114B67
:10FBC00000204FF4806500BF00EB800413F8246030
:10FBD00096B903EB84063489768914443444A4B27C
:10FBE000AC4209D2088000EB800003EB8000418921
:10FBF00011444181002070BD401C80B20228E3D333
:10FC0000072070BDA42B0020111213140D0E0F102D
:10FC10000C2500202C250020582500200D00030075
:10FC2000F98202000E000300F98202000F000300B7
:10FC3000F982020010000300F982020007000000B0
:10FC400000000000000000000000000000000000B4
:10FC5000060000000000000000000000000000009E
:10FC60000000000010000000000000000000000084
:10FC70000000000000000000110000000000000073
:10FC80000000000000000000000000000100000073
:10FC9000010001008CFC020001000100A0FC020038
:10FCA0000000000085DA0200E1960200770A0000F9
:10FCB00000000000770A0000000000007ADA00006F
:10FCC00000000000F1D0020007000000000000006A
:10FCD00000000000000000000000000085DB0200C2
:10FCE00079EB0200FD99020061970200010000001B
:10FCF00000000000010006008422002005EC020044
:10FD000001000000000000000000000000000000F2
:10FD100000000000070000000000000000000000DC
:10FD200000000000000000000300000000000000D0
:10FD300000000000000000000000000005000000BE
:10FD400000000000000000000000000000000000B3
:10FD5000ADDE020050EADA308883B89F604F15F3B9
:10FD60000000C98E0000005015C8020071CA0200D0
:10FD700003000000C4290020000000000000000073
:10FD80000338FDD870470000FC2200200000FFFF70
:10FD9000DEC0ADDEFF011EF1DEC0ADDEFE011EF1F4
:10FDA00030313233343536373839414243444546B1
:10FDB0006E72665F6673746F726167655F696E69A4
:10FDC00074006E72665F6673746F726167655F75EB
:10FDD0006E696E6974006E72665F6673746F7261CD
:10FDE00067655F72656164006E72665F6673746FEB
:10FDF000726167655F7772697465006E72665F66CF
:10FE000073746F726167655F65726173650000008E
:10FE1000402300200010000004000000010000004A
:10FE2000C59D020045F502008DE1020019F80200AF
:10FE3000B58D020055E4020015F8020049A0020049
:10FE4000F4090300F80903000000000000000000AE
:10FE500000000000000000007C2C002040FE02009A
:10FE600058FE020004000000556E6B6E6F776E2026
:10FE70006572726F7220636F64650000000000009D
:10FE80002806030001000000D40403000200000063
:10FE9000C80203000300000048050300040000003E
:10FEA0009C050300050000007C0403000600000020
:10FEB0001804030007000000840503000800000088
:10FEC0009004030009000000F40403000A0000008D
:10FED000100603000B000000B00203000C0000003D
:10FEE000A80403000D000000780603000E000000C7
:10FEF000740503000F000000B005030010000000AF
:10FF0000E4050300110000008C060300120000004D
:10FF10006006030013000000FC05030080000000E1
:10FF200030040300810000006C0303008200000025
:10FF30002C030300830000000C0303008400000076
:10FF400048030300850000005404030086000000FD
:10FF50005C05030090000000F8030300910000001E
:10FF6000EC02030092000000BC04030000820000C9
:10FF7000C405030001820000100503000282000096
:10FF80002C050300008400008803030001840000A6
:10FF90003406030002840000D00303000384000041
:10FFA000AC030300C5B9020099B9020091B902007F
:10FFB000FFFFFFFFFFFFFFFFFFFFFFFFFFFFFFFF51
:10FFC00000000000000000000000D6010701000052
:10FFD000400A0300480A030000000000000000007F
:10FFE00001000007D0FF0200E0FF0200080000004F
:10FFF00008000300180003000800000018000300B8
:020000040003F7
:100000002800030008000000780A0300900A03009B
:100010000000000000000000680A0300780A0300E6
:100020000000000000000000F8090300000A0300BF
:10003000000A0300280A0300280A0300380A030004
:10004000380A0300400A0300282200202800030089
:100050004800030008000000480A0300580A030093
:10006000580A0300680A03005800030068000300F0
:1000700008000000004040404040404040404141B6
:10008000414141404040404040404040404040406D
:100090004040404040050202020202020202020207
:1000A0000202020202202020202020202020200204
:1000B0000202020202029090909090901010101094
:1000C0001010101010101010101010101010101030
:1000D00002020202020288888888888808080808C4
:1000E0000808080808080808080808080808080890
:1000F00002020202400000007500030073645F62A8
:100100006C655F6761705F646174615F6C656E6789
:1001100074685F7570646174652829202872657140
:100120007565737429206F6E20636F6E6E656374DE
:10013000696F6E20307825782072657475726E65EF
:10014000642025732E000000546865207265717567
:10015000657374656420636F6D62696E6174696F45
:100160006E206F6620545820616E642052582070B3
:1001700061636B6574206C656E6774687320697366
:1001800020746F6F206C6F6E672062792025752058
:100190006D6963726F7365636F6E64732E00000028
:1001A00054686520626F6F746C6F6164657220685B
:1001B00061732077726974652070726F74656374FF
:1001C0006564206974732073657474696E67732045
:1001D000706167652E20546869732070726F68695A
:1001E000626974732073657474696E6720746865DE
:1001F000207065657220646174612E2054686520EA
:10020000626F6F746C6F61646572206D75737420BA
:10021000626520636F6D70696C65642077697468CE
:10022000204E52465F424C5F53455454494E47530B
:100230005F504147455F50524F544543543D302035
:10024000746F20616C6C6F772073657474696E676E
:1002500020746865207065657220646174612E0089
:10026000616464725F69735F77697468696E5F6205
:100270006F756E647328705F66732C20706167659C
:100280005F616464722C20286C656E202A20705F88
:1002900066732D3E705F666C6173685F696E666F32
:1002A0002D3E65726173655F756E69742929000062
:1002B0004E52465F4552524F525F494E56414C494D
:1002C000445F4441544100004E52465F4552524FF4
:1002D000525F534F46544445564943455F4E4F5431
:1002E0005F454E41424C4544000000004E52465F7F
:1002F0004552524F525F464541545552455F4E4F0D
:10030000545F454E41424C45440000004E52465F0A
:100310004552524F525F4D555445585F554E4C4FC4
:10032000434B5F4641494C45440000004E52465FF6
:100330004552524F525F4D555445585F4C4F434BB9
:100340005F4641494C4544004E52465F4552524F2C
:10035000525F4D555445585F434F4E445F494E4997
:10036000545F4641494C4544000000004E52465FF0
:100370004552524F525F4D555445585F494E49546E
:100380005F4641494C4544004E52465F4552524FEC
:10039000525F424C455F495053505F52585F504B3B
:1003A000545F5452554E4341544544004E52465FAB
:1003B0004552524F525F424C455F495053505F5037
:1003C0004545525F52454A454354454400000000AC
:1003D0004E52465F4552524F525F424C455F495024
:1003E00053505F4C494E4B5F444953434F4E4E452B
:1003F00043544544000000004E52465F4552524F60
:10040000525F4150495F4E4F545F494D504C454DEE
:10041000454E5445440000004E52465F4552524FEF
:10042000525F4E4F545F535550504F525445440005
:100430004E52465F4552524F525F4D4F44554C45C8
:100440005F4E4F545F494E495449414C495A4544C7
:10045000000000004E52465F4552524F525F4D4FD2
:1004600044554C455F414C52454144595F494E49C2
:100470005449414C495A4544000000004E52465FE1
:100480004552524F525F4E4F545F464F554E4400B7
:100490004E52465F4552524F525F494E56414C496B
:1004A000445F5354415445004E52465F4552524FAB
:1004B000525F444154415F53495A45004E52465F92
:1004C0004552524F525F494F5F50454E44494E4747
:1004D000000000004E52465F4552524F525F535645
:1004E000435F48414E444C45525F4D495353494E3A
:1004F000470000004E52465F4552524F525F494EF0
:1005000056414C49445F4C454E475448000000005A
:100510004E52465F4552524F525F4452565F5457B7
:10052000495F4552525F414E41434B004E52465F38
:100530004552524F525F4452565F5457495F45529D
:10054000525F444E41434B004E52465F4552524F1C
:10055000525F494E5445524E414C00004E52465F48
:100560004552524F525F53544F524147455F465593
:100570004C4C00004E52465F4552524F525F4E5512
:100580004C4C00004E52465F4552524F525F494E0E
:1005900056414C49445F504152414D004E52465FD6
:1005A0004552524F525F4E4F5F4D454D0000000087
:1005B0004E52465F4552524F525F464F5242494457
:1005C00044454E004E52465F4552524F525F445290
:1005D000565F5457495F4552525F4F5645525255E8
:1005E0004E0000004E52465F4552524F525F494EF8
:1005F00056414C49445F4144445200004E52465FCC
:100600004552524F525F5245534F55524345530046
:100610004E52465F4552524F525F494E56414C49E9
:10062000445F464C414753004E52465F5355434347
:10063000455353004E52465F4552524F525F424C13
:10064000455F495053505F4348414E4E454C5F41D2
:100650004C52454144595F4558495354530000009A
:100660004E52465F4552524F525F434F4E4E5F438C
:100670004F554E54000000004E52465F4552524FB7
:10068000525F54494D454F55540000004E52465F4D
:100690004552524F525F4255535900007761726E76
:1006A000696E670064656275670000001B5B313B23
:1006B00033306D001B5B306D000000001B5B313B75
:1006C00033316D001B5B313B33326D001B5B313BC3
:1006D00033336D001B5B313B33346D001B5B313BAF
:1006E00033356D001B5B313B33366D001B5B313B9B
:1006F00033376D00696E666F000000006572726FBF
:100700007200000073645F626C655F6366675F73AD
:10071000657428292072657475726E65642025736E
:10072000207768656E20617474656D7074696E679A
:1007300020746F2073657420424C455F47415454C8
:10074000535F4346475F534552564943455F4348CD
:10075000414E4745442E000073645F626C655F63E1
:1007600066675F73657428292072657475726E659B
:1007700064202573207768656E20617474656D70E0
:1007800074696E6720746F2073657420424C455FF6
:10079000434F4D4D4F4E5F4346475F56535F555550
:1007A00049442E0073645F626C655F6366675F73C4
:1007B000657428292072657475726E6564202573CE
:1007C000207768656E20617474656D7074696E67FA
:1007D00020746F2073657420424C455F4741545428
:1007E000535F4346475F415454525F5441425F5305
:1007F000495A452E0000000073645F626C655F63B8
:1008000066675F73657428292072657475726E65FA
:1008100064202573207768656E20617474656D703F
:1008200074696E6720746F2073657420424C455F55
:10083000434F4E4E5F4346475F4741502E000000F6
:1008400073645F626C655F6366675F7365742829B4
:100850002072657475726E656420257320776865F3
:100860006E20617474656D7074696E6720746F209A
:1008700073657420424C455F4741505F4346475F74
:10088000524F4C455F434F554E542E006E72665F7B
:10089000626C655F6761747400000000636C6F6375
:1008A0006B000000434C4F434B0000004750494F42
:1008B000544500005052530055415254000000006E
:1008C000554152544500000061746669666F2E6D93
:1008D0005F717565756500006E72665F6673746F33
:1008E000726167650000000061746669666F2E6D55
:1008F0005F6669666F0000007077725F6D676D7488
:100900000000000062616C6C6F632E6C6F675F6D3E
:10091000656D706F6F6C0000617070006E72665F65
:10092000736468006E72665F7364685F626C650012
:100930006E72665F7364685F736F6300900A030092
:10094000282200200C02000020650200F00A0300AB
:10095000342400209C2D0000FC6A02008C08030057
:10096000000003039C08030000000000A40803002B
:1009700000000000AC08030000000000B408030001
:1009800000000000B808030000000000C0080300D9
:1009900000000000C808030000000003D80803009E
:1009A00000000303E808030000000003F808030048
:1009B0000000000004090300000000031809030000
:1009C000000003031C0903000000030324090300C3
:1009D00000000303300903000000030390230020FC
:1009E0008823002090230020E82C002020240020D1
:1009F00018000000A56D0200398002000000000010
:100A0000A9AB0200342400208B740200542400207F
:100A1000CD7E0200000000003D7F020000000000CB
:100A20003D810200000000002BAD020048240020A0
:100A3000797B02009C280020657E020000000000F7
:100A400045B402000000000021EF02000000000099
:100A50007DB4020000000000F57402005424002060
:100A6000797C02000000000099C202000000000032
:100A700025C40200000000005D87020000000000A5
:100A80005DE50200000000005DB40200000000000F
:100A9000062BFFFF0A1801042D81DA022A180179BA
:100AA00009390A01711310240240200A1A1844124D
:100AB00020AA40080425A4FF0214FC06031A9C0483
:100AC0001AF4041AA4041AB4041AAC041ABC041AC2
:100AD000C4041ACC041AD4041ADC041AE4041AEC70
:100AE00004515B90D009210B245D946C012400001B
:020000040007F3
:10F00000D29BC57601000000010000000100000055
:10F010000000000000000000F0AA0000C4CD651C44
:10F0200001000000000000000000000000000000DF
:10F0300000000000000000000000000000000000D0
:10F0400000000000000000000000000000000000C0
:0CF05000000000000000000000000000B4
:00000001FF
